:020000040800F2
:10500000701C0020D5500008ED8E00083185000886
:105010000000000000000000000000000000000090
:10502000000000000000000000000000659A000879
:10503000000000000000000005970008A19B000888
:10504000E7500008E7500008E7500008E750000864
:10505000E7500008295F0008E7500008E750000803
:1050600000000000E7500008015C0008E75000085D
:10507000E7500008DD8A000800000000E750000843
:1050800000000000E75000080000000000000000E1
:10509000E750000800000000E7500008E750000853
:1050A000E7500008E7500008E750000815A6000880
:1050B000E7500008E7500008000000000000000072
:1050C0000348854600F0E8FC0048004789B900081D
:1050D000701C00200448804704480047FEE7FEE7B4
:1050E000FEE7FEE7FEE7FEE73D9C0008C150000832
:1050F00030B50B46014600202022012409E00D4670
:10510000D5409D4205D31D469540491B25469540F7
:1051100040191546521E002DF1DC30BDF0B51FB40C
:105120000646002082B005464024019100901BE015
:10513000019922460F46304600F098FB049A059BE1
:10514000801A994110D310461946224600F07EFB82
:10515000361A8F410197224601200021009F00F05E
:1051600075FB38184D4100902046641E0028DFDC96
:10517000019B00982946324607B0F0BD03460B4319
:105180009B0703D009E008C9121F08C0042AFAD2FD
:1051900003E00B780370401C491C521EF9D2704783
:1051A000D2B201E00270401C491EFBD270470022BF
:1051B000F6E710B513460A4604461946FFF7F0FF16
:1051C000204610BD30B504460020034600E05B1CBD
:1051D000934203D2E05CCD5C401BF8D030BDF8B503
:1051E00002464A40D40F42004B0052085B089A42E4
:1051F00002D20246084611464A0023D0C30D4A0097
:10520000DDB2120EAD1A202D35DA49020126490A07
:10521000F6058A19002C00D0524220214F1B11465E
:10522000B9402A411018C20D9A4221D0002C17D043
:10523000012D08DCDA05801AD20F8019D207DBB203
:1052400000F040FBF8BDDA05801A012340001B0680
:10525000C01880185A428018CA0F1043490007E04E
:105260004908C2071143DA05801A801940088018DE
:1052700000F020FBF8BD61000122511A001BF7E786
:105280000122D2075140AAE70122D2075040A6E7E7
:1052900070B502464A40D50F40004A00ED0740086D
:1052A0005208002814D0002A12D0C40DD30D410298
:1052B0000120C0055202490A520AE41A09181218BC
:1052C0007D34914201D3641C00E04900002C01DAD6
:1052D000002070BD0023914201D3891A0343400886
:1052E00049000028F7D100290AD0914202D10121BA
:1052F000C90705E0914201D2012101E00121C94322
:10530000E005C018401900F0D5FA70BD420005D084
:105310004200120E52428A4201DB00207047C9054A
:1053200008187047F0B507460846584087B0C00FC8
:10533000049048000E46590040084908BC1A8841AC
:1053400005D2384631461E4617460B4602465800DF
:10535000400810434CD0300D039040055900400DDB
:10536000490D0590401A0290402872DA1803012175
:10537000000B09050843019004980092002805D00D
:1053800001995242002088410092019002984021E8
:105390000A1A0199009800F059FA05460C466B4626
:1053A00007CB00F074FAC0197141039A0E0D002367
:1053B000D71756401A467A40164344D0049A002A1A
:1053C0002DD0029A012A039A15DC1205C01A9141C8
:1053D00001263605001C7141D20F059ED2070093AD
:1053E000019202962A46234600F0B2FA07B0F0BDB9
:1053F00038463146FAE71605224A0F46B218C01A57
:10540000B74101210905001C4F4100187F41114699
:1054100018187941E20F10436D19644113E0E20757
:105420006D0815436408C2071443039A0126120548
:10543000C01A91413605001C7141CE074008304327
:105440004908C01851412A46234600F074FACDE7B6
:10545000FFE7049801224000C117121A00238B4174
:1054600004983146C417381AA141EEE730B401243C
:10547000E407634030BC55E730B40124E4076140E1
:1054800030BC4FE70000E0FFF0B51FB488B00B99C7
:105490000998002448400999C00F4900490809911A
:1054A000C0070B990090490049080B910999089889
:1054B000A64608431CD00B990A98084318D00998AF
:1054C00001244000420D4800410D099824050003C5
:1054D000000B204309900B980003000B20430B9016
:1054E00050181C494018002201901446104605E04F
:1054F000002001460DB0F0BD032801DA034600E0AC
:1055000003239C46C11A0AAE0AE05F0008ADED5BBA
:105510004F00F75B7D430027AA187C41491C5B1EA6
:105520006145F2DD410004AB5A522104120C0A43DA
:10553000240C401C0828DFDB01980290009970467B
:1055400001910090059B049A0799069800F000FAD3
:10555000D0E700000DFCFFFFF0B50C465C4085B0C5
:10556000E40FE40703944C000026640859009446B5
:10557000490802460296224321D062460A431ED0C1
:105580006200570D4A000E032303550D0124024605
:105590002C492405781B1B0B360B4018234326434C
:1055A000614600901C46501AB44103D30098401C39
:1055B000009002E0921800985B41002803DA002076
:1055C000014605B0F0BD00200121090507468646C9
:1055D00011E064461D46141BB54106D36546521BB7
:1055E000B341744607430C43A646CD07400849081B
:1055F000284392185B4105460D43EAD110461843F3
:1056000013D06046194650407140084306D06046AA
:10561000101AB34106D20122002306E00022012322
:10562000DB0702E00122D2435310009874460105C3
:10563000381C6141029C039D0019694100F07BF90F
:10564000BFE70000FD03000070B54B005B0803439B
:105650000BD04B005C0D002633466542B341D41796
:10566000AD1AA34102DB0020014670BD12053018BF
:10567000514170BDC217C10F504010B54018CA0744
:105680009623002100F01EF910BD10B500229623CC
:10569000114600F017F910BD0EB5C217C10F5040EA
:1056A000CA0740180021054B0293019200910A4657
:1056B0000B4600F04DF903B000BD000033040000BC
:1056C0000EB505490291002100910A460B46019151
:1056D00000F03EF903B000BD330400004100400279
:1056E0000122400AD205090E80187F2901DA002024
:1056F0007047962903DC9622511AC84070479639A4
:105700008840704770B5CD0F4A0009030123090B8B
:105710001B0519430B4BED070024520D9A4201DA89
:10572000002070BD074B34339A4203DC9A1A00F014
:105730009DF802E00449511888402C43F1D04042C2
:1057400070BD0000FF030000CDFBFFFF4A0009030E
:105750000123090B1B051943094B10B5520D9A4241
:1057600001DA002010BD064B34339A4203DC9A1A4A
:1057700000F07CF810BD03495118884010BD0000AE
:10578000FF030000CDFBFFFFC20FD207400040081F
:105790000BD0C10D0723DB01C91840020905400ADF
:1057A0001143C2084007114370470020014670476B
:1057B00010B5002904DB0124E40740428C41214656
:1057C000002B04DB1C460123DB075242A3418B4222
:1057D00000D1824210BD000010B5002904DB012475
:1057E000E40740428C412146002B04DB1C46012388
:1057F000DB075242A341994200D1904210BD000004
:10580000CB0FDB07490010B5490802460A4307D011
:105810000A0D07240903E401090B121B002A01DC0D
:10582000002010BDC900440F0C43C100E018D20590
:10583000801800F03FF810BD0122D207002800DBDD
:10584000101A002900DB511A8142704710B5202A36
:1058500004DB0146203A9140002010BD91402023F6
:105860009C1A0346E3401943904010BD10B5202A0E
:1058700004DB0846203AD040002110BD0B46D3403F
:10588000D0402024A21A91400843194610BD10B5FB
:10589000202A06DBCB170846203A1041C1170B43DC
:1058A00006E00B461341D0402024A21A9140084341
:1058B000194610BD002904DA401C490001D14008F6
:1058C0004000704770B40024050C05D1102400047A
:1058D00002D1002921D01124050E01D10002083483
:1058E000050F01D10001241D850F01D18000A41CEA
:1058F000002801DB4000641C002908D020252E1B55
:105900000D46F540A14000D001212943084301067E
:105910001B1B000ADB1D02D5002070BC7047DB0595
:10592000181880180029F8DA401C4900F5D170BC1D
:1059300040084000704710B5002B08DA0024401CD6
:10594000614192185B411A4301D14008400010BDEB
:10595000F0B51FB482B005460C0003D0084604F031
:105960000DFF02E004F00AFF2030024600902146BD
:105970002846FFF76BFF049B059A04460F46184321
:105980001143084314D0184610431BD000984021FF
:105990000A1A18460599FFF769FF05460E46009A50
:1059A00005990498FFF752FF084305D0012004E051
:1059B0002046394607B0F0BD0020C11705430E430D
:1059C0002C43374300990E986305401A7905E40A81
:1059D00000220C43FD0A0A3002D500200146E9E707
:1059E0000105101969410C9C0D9D00196941FFF7D3
:1059F000A2FFDFE7FEB500231A461B1A8A4103DB2C
:105A00000020014603B0F0BD4A000D0301212D0B1B
:105A10000905520D0D43D10702D100186D41521EE8
:105A20005110FF31FF310131002704463E46384610
:105A3000009701910246012100200905FFF716FF9A
:105A4000C3197141F818324684468E464A41614670
:105A50002846611A904104D36046241A954176463F
:105A60001F46241900986D41401C00903428E1DD48
:105A7000F91930467041091BA84103D20022D243D4
:105A8000134601E00022134601980105381C7141BC
:105A9000FFF751FFB6E70000064C0125064E05E072
:105AA000E36807CC2B430C3C98471034B442F7D33F
:105AB000FFF70AFB78C8000898C8000870B58C1872
:105AC0000578401C6B075B0F01D10378401C2A113D
:105AD00006D10278401C03E006780E70401C491C79
:105AE0005B1EF9D12B0705D40023521E0DD40B7079
:105AF000491CFAE70378401CCB1A921C03E01D787E
:105B00000D70491C5B1C521EF9D5A142D8D3002050
:105B100070BD000038B50446064805490068FFF727
:105B2000E7FA604300E0401E00900028FBD138BD3A
:105B300040420F0064010020F8B504460068816807
:105B40008907890F012902D10168C90722D181681B
:105B5000114A10261140012500290ED181682943E0
:105B600081600120FFF7D6FF01F050F907460CE0F5
:105B700001F04CF9C01B0A2807D9606D30436065FD
:105B8000A06D2843A0650120F8BD20680068C043CF
:105B9000C007EDD10020F8BD170000801FB50B48ED
:105BA00000900B4801900B4802900B480390694607
:105BB0000A4805F0D9F90A4A08481146083905F09B
:105BC000C1F800F097FB002004B010BD81C60008AA
:105BD0005DC60008BDC60008BBC6000870010020F5
:105BE0001000002010B500231A4603E0845CE3187F
:105BF0009BB2521C8A42F9D3D84380B210BD000038
:105C000010B5034800F0BEFE024800F0BBFE10BD18
:105C10000C180020C417002030B5446C1C252C4003
:105C20000125A540046C6560046863608368102BDF
:105C3000036803D099600068C26030BD9A60006854
:105C4000C16030BDF0B58BB000200790874E0A20B0
:105C500005F03AFD7D20400105F050FD844C002503
:105C6000206C401C206483480990FF3881380890DC
:105C70000021804861710B30226CC270120A0272DE
:105C800081740A2141727C4909788172218D0173E6
:105C900045707A4909980A780274497841747549BF
:105CA0001C2000220B3105F0F9FD607906214843E4
:105CB00000211C3005F004FE022005F055FD704F58
:105CC00000210F2005F080FC38426064F8D0606C41
:105CD000411C16D040047DD58122D20100210F2025
:105CE00005F0B1FD0021102005F06EFC4106490EC3
:105CF0000022644805F09EFC624F787A022802D0A8
:105D00009FE004F0AFFD02225C49781DFFF75AFACC
:105D100000287DD105F025FE554A803203C205F0EA
:105D20000DFE534A8032D160906002900798039133
:105D300000281AD101205349079053482839CB8EA7
:105D40000380098F514AFF31C33189B2E184914206
:105D50000BD952428918E1845B1C4C4A99B20B3230
:105D60000180914201D300210180424B69000B3335
:105D70000898CA18017A0A91D174407A049041496E
:105D8000107528394A8E68468280898EC180042227
:105D9000791C581CFFF7F2F90198B04205DA064663
:105DA00069460A9808750498487532480C210B30EA
:105DB00041722F4F4B2202998037D204039800235F
:105DC000891858410206080A1043019005F075FC35
:105DD000019800E048E040084000010E00027961AF
:105DE000386124480CCF1530083F05F08FFD21485D
:105DF000FB681930BA6805F089FD1E487B691D30C3
:105E00003A6905F083FD1B4900220B31192000E09F
:105E100017E005F043FD0021192005F051FD012098
:105E200005F0A2FC0006000E607305D100210F20D2
:105E300005F0CAFB0006F9D5802200210F2005F0ED
:105E400002FD6D1CEDB20A2D00D211E70748864213
:105E500008D0002E06D00020A073022020706846D3
:105E6000808A60850BB0F0BD094AE6E7FFFF0100BC
:105E700070000020691400202C0100204001002047
:105E800000D02724F01200204C010020E70300007E
:105E9000009027241449012048720A4602205E32ED
:105EA000507203203C3A507204200E3A50720F4850
:105EB0000D4B0078087022310870203108770C49AA
:105EC0005A1C08785871497899712333187159719F
:105ED000203318775977107551751A461E32107590
:105EE0005175107651767047C81100201E010020B0
:105EF0004001002010B503F08BFD202003F046FE8A
:105F0000012005F09BFA002003F040FE044805F054
:105F100039F9044805F0E8FB002005F01DFC10BD30
:105F20000801002083800000F8B503F03DFE052045
:105F30000121000700F056FF0025144C002800D076
:105F40006560134E0221304600F04CFF002815D149
:105F5000012020700F48808F00280ED00127BF023B
:105F600000223946304600F04AFF0A2004F05AFE6B
:105F700001223946304600F042FF6560012000F002
:105F800069FE022000F066FEF8BD0000500100200E
:105F900000040050C80D00207047000010B50849EB
:105FA00000224A6107494B684C1523434B604B68FC
:105FB000082423434B60C009C001026010BD0000EB
:105FC00054180020002002407FB500250C460646EC
:105FD000039500F00FFEE009029003A901960095D9
:105FE000684600F09FFD002804D000F0D7FD002097
:105FF00004B070BD00F0D2FD0120F9E710B5002318
:1060000002E0C45CCC545B1C9342FAD310BD000088
:1060100010B5214A00219069C305204804D5416983
:10602000022319434161911593699B0505D5436985
:106030000124234343616302194393695B0505D53A
:106040004369082423434361E301194393691B0512
:1060500005D54369042423434361630219439369CB
:106060009B0405D54369102423434361630219430C
:1060700093699B0304D5446920231C43446119435D
:106080009369DB0305D54369402423434361A002A0
:106090000143916110BD000000200240541800200F
:1060A00070B5054600F0B2FE0646184C0AE0681CC2
:1060B00008D0002D04D000F0A9FE801BA84201D911
:1060C000032070BDA069C007F1D1A069800701D588
:1060D0000220A061A069C00511D4A06980050ED47A
:1060E000A06940050BD4A069000508D4A06980040C
:1060F00005D4A069800302D4A069C00303D5FFF7CB
:1061000087FF012070BD002070BD0000002002400C
:10611000F8B51746002605460C4600F06BFD09E071
:1061200029460220226800F047FD002804D1241DE2
:106130002D1D361DBE42F3D300F030FDBE4201D20C
:106140000020F8BD0120F8BD10B508490246002026
:10615000054B497905E044001C5B944203D0401C88
:10616000C0B28842F7D310BD861300207000002013
:1061700010B500F03CFE10BD10B5094801F05CF808
:1061800080B2FFF79DFA074A074BFFF77DF900221F
:10619000064BFFF7E1F9FFF7D9FA80B210BD000016
:1061A00078160020F853E3A59B843E4000408F40C2
:1061B00070B50024204603F03DFA47494748A20045
:1061C000641CE4B28150142CF9D3464944480A7A3D
:1061D0000275497A417544490A78027649784176D0
:1061E0003F490520133148720A2005F06DFA7D20E1
:1061F000400105F083FA3A49002213310C2005F0E2
:106200004DFB00210C2005F05BFB384801F014F831
:10621000344C0125223CA085AD0309E0334801F050
:106220000BF880B2A085618FFF392D39884206DBDB
:10623000618F80B28842F1D349198842EED802209A
:1062400005F092FA002003F0F5F9294D00210F2006
:1062500005F0BAF928426064F8D0606C411C38D06F
:10626000400435D58122D20100210F2005F0EBFA40
:106270000021102005F0A8F941061948490E002216
:10628000C73005F0D7F9164DC735687A05281FD1F4
:1062900002221549681DFEF795FF002818D1114804
:1062A000AE7C66710422691C3A30FEF767FF29460E
:1062B0001331084672000D468330FEF75FFF6079A8
:1062C0002946420005484A38FEF758FF032020704F
:1062D00070BD04F0C7FA0000FFFF0100E8130020C2
:1062E0002912002092000020400100207816002092
:1062F00000D0272410B5144C144822461032114601
:10630000083904F01FFD0022114BE168A068FFF777
:1063100023F9104A104B05F043FC00220F4BFFF706
:10632000ABF800220E4BFFF7AFF8FFF769FA2060D9
:1063300000221346E168A068FFF73AFA01D020680E
:1063400010BD0020206010BD000000207001002062
:1063500000AA8F406C45D9CC955BC83F0000F03F48
:1063600040A5E54010B5084800F096FA0A21064815
:1063700000F032FA044800F01DF9800503D5024808
:1063800000F01AF980B210BD1C160020F8B52F4D90
:1063900000220121284600F032FDFFF7E3FFFFF75E
:1063A00074F92B4E3146FEF773FF2A4C0122A06090
:1063B0001146284600F023FD2749A06800258842A1
:1063C0003EDB2078254F002815D02570FFF7CAFF47
:1063D000FFF75BF93146FEF75BFFA060FFF7D4F9EA
:1063E00000223B46FFF742F800221D4BFFF74CF816
:1063F000FFF706FA6060A068FFF7C6F900223B4687
:10640000FFF734F8174A184BFFF73EF806460F46D9
:106410006068FFF7B9F9134A144B5242FFF734F89A
:1064200032463B46FEF77EFFFFF7EAF9104960600F
:10643000884201DD616004E0FF21C905C84200D344
:1064400065606068FFF74AF9C0B2F8BD000400500B
:1064500000401B44480000200000604000000C4049
:1064600000E064403333333333B33040CCCCEC3FC3
:106470000000C842F8B5054604464035287C002691
:10648000012808D001202874206881688907890FB5
:1064900001290ED101E00220F8BD0168C90708D02A
:1064A000606D202108436065012600202874304675
:1064B000F8BD616DFF2201329143022211436165F3
:1064C000C1688907890F0091C16889088900C16086
:1064D0002068816892071143816000F097FC0746AD
:1064E0000EE000F093FCC01B0A2809D9606D022160
:1064F0008843102108436065002028740120F8BDFE
:10650000206880680028ECDB2068C168009A11438D
:10651000C160606D80088000401C6065C5E70000B8
:10652000F8B506460D464036317C01290DD00121D3
:10653000317401688A68520709D5416D20221143E0
:106540004165002030740120F8BD0220F8BD174BD2
:106550006A68D80547109A42154C8A6A2B6812D08F
:106560005B035B0B1A438A622968490305D5A1685E
:106570000143A1600A20FFF7CDFA2868800312D5F5
:10658000A06838430EE05B035B0B9A438A6229687C
:10659000490302D5A1688143A1602868800302D520
:1065A000A068B843A06000203074F8BD011000005E
:1065B00000270140406D70470068006C7047000084
:1065C00070B5040006D0606D2646002540360028D0
:1065D00002D006E0012070BDA5653574204600F0AC
:1065E000D3F8606DC00603D421688868400705D5DC
:1065F000606D1021084360653574EBE7606DFF2224
:106600000132904302221043606588688207920F2E
:106610005B48012A02D10A68D2072BD103236268A2
:106620009B079A4205D05B429A4202D05B009A4295
:1066300009D10A69920092080A6121680A696368AF
:106640001A430A610CE00A69920092080A618168A3
:106650000F229204914381608168626811438160D6
:106660002168CA6818239A43CA602168CA68A36867
:106670001A43CA6081680122520691438160816891
:10668000A28E52061143816020688168C90004D43B
:10669000816801221207114381602068C168394A6C
:1066A0001140C1602069E168022825D00020014323
:1066B000204620300278037B52035B001A431143CB
:1066C000226B1143A26992031143E269D203114381
:1066D0002268D3681943D160616A0A46FF3AC23A18
:1066E00005D0A26A11432268D3681943D160427869
:1066F0000121012A02D00BE00420D8E7007800280D
:1067000023D0606D202210436065A06D0843A06512
:10671000E06B012820681FD00169C90703D0016917
:1067200049084900016120684169C908C9004161FF
:1067300020684169A26B11434161A565606D8008C5
:106740008000401C6065002070BD2068C268012385
:106750001B041A43C260DBE70269FF239B009A43D4
:10676000026120680269236CA66C1A43636C334390
:106770001A430261206802690A430261D3E70000FC
:10678000002701401902FEFF10B586B0044614210F
:106790006846FEF70CFD0E492068884216D10D4868
:1067A000416B421511434163C16A01221143C16229
:1067B000C06A6946104005900220009003200190B5
:1067C000002002900520000700F050FA06B010BD2E
:1067D0000024014000100240F8B5044640692546F7
:1067E00040350E4608280BD02068C068C00709D085
:1067F000606D202108436065002028740120F8BDE9
:10680000082700E00C2700F001FB009011E0701C4D
:106810000FD0002E05D000F0F9FA0099401AB042CE
:1068200007D9606D042108436065002028740320A7
:10683000F8BD206800683842E9D0606D0121490246
:10684000084360652068C16809058A0F0C21002A89
:106850001BD12022125D002A17D10268120714D51D
:10686000826853070122002B08DB43688B43436097
:10687000606D130298431043606506E0606D20234D
:1068800018436065A06D1043A065A069002801D180
:10689000206801600020F8BD70B504462168002022
:1068A0008968490721D425464035297C01291CD017
:1068B00001212974E169012904D02046FFF73CF940
:1068C000002811D1616D0A4A1140FF2201321143A3
:1068D00061650021A165297422681C21116021686D
:1068E0008A6804231A438A6070BD022070BD0000CC
:1068F000FEF1FFFF30B5014620314A790023022A1C
:1069000004D00422C2630B71012030BD02681468F8
:106910000E25AC43146002681468640864001460B7
:10692000446C1C22144001221546006CA5404560B1
:106930004A7118460B7130BD70B5002401462031F4
:106940004A79022A03D00421C163012418E00268B5
:1069500013680E25AB431360026813685B085B0085
:106960001360436C1C221340012215469D40036CAA
:106970005D604A7100220A71816B002900D088474E
:10698000204670BDF0B4016C0D6801680C68466C5F
:106990001C2304221E401746B7402F420ED0670723
:1069A0000CD50C68A40602D40C6894430C60416CAE
:1069B00019408A40016C4A60016B1AE00227B74017
:1069C00002462F402032002F17D0A70715D50C689C
:1069D000A40605D40C680A25AC430C600121517152
:1069E000446C02211C40036CA140596000211171CC
:1069F000C16A002918D0F0BC08470827B7402F42C9
:106A000012D0240710D50C680E25AC430C60446CE2
:106A100001211C400B46A340046C6360C1635171AB
:106A200000211171416BE4E7F0BC704770B50400C0
:106A30003CD01F48256814212818FEF759FB800018
:106A400060641C48206402212046203002464171C7
:106A500029681948E3680140A068666918432369FA
:106A600033431843A3691843E3691843236A18435F
:106A7000084328600121A0688903884210D00D488E
:106A80008030836A656C1C210D400F26AE40B343F5
:106A90008362656C63680D40816AAB400B4383621F
:106AA0000020E06301215171107170BD012070BDA3
:106AB000F8FFFDBF000002400F80FFFFF8B504465D
:106AC0008C46203001790025012909D00126067164
:106AD00041790027012905D0077102252846F8BD14
:106AE0000220F8BD02214171E7632068016849086E
:106AF0004900016061462046FFF78EF8206B0028B0
:106B00002068016801D00E2205E004229143016053
:106B1000206801680A22114301602068016831433E
:106B20000160DBE7F8B51A4E0546307C0F460128B8
:106B300007D0012030741748FFF7B2FA010002D0E5
:106B400021E00220F8BD0020C04338606C6814E0EA
:106B50002046FFF723FA0F48FFF7A2FA01460E4836
:106B6000426808239A434260426843159A43426050
:106B7000002901D03C6006E08034A8686A68C00142
:106B80008018A042E4D8002030740846F8BD000008
:106B90005418002050C300000020024005484168FE
:106BA00002221143416041680122114341600020EB
:106BB0007047000000200240F8B50C4C1646207CBF
:106BC0000F46012808D0012020740948FFF768FA11
:106BD0000025002802D006E00220F8BD65613E6075
:106BE0000348FFF75DFA2574F8BD00005418002033
:106BF00050C3000011484168C9070BD0EFF3108162
:106C000072B60F4AC2600F4AC26081F310884168B1
:106C1000C9070ED1416889070DD5EFF3108172B60F
:106C2000094A0261094A026181F3108840688007BD
:106C300001D501207047002070470000002002406D
:106C4000EFCDAB8905040302BFAE9D8C161514135E
:106C50007047000010B504494A69024202D04861F9
:106C6000FFF7F6FF10BD000000040140FCB5002353
:106C70000124A2E027462A469F403A406FD04D6843
:106C8000012D05D0022D03D0112D01D0122D16D1CA
:106C900085680326AC465D00AE46AE406546B5430A
:106CA000AC46CE687546AE4065462E438660466863
:106CB0000D79BE43ED06ED0F9D4035434560C66836
:106CC0005F000325BD40AE46AE4335468E68BE40EC
:106CD0002E43C6604E68022E01D0122E14D1DE085B
:106CE000B60036180196366A5D07B446EE0E0F25DB
:106CF000B54000966646AE43B4460D69009EB54069
:106D000066462E43019D2E6206687546AE430D7998
:106D1000AD07AD0FBD40354305604D68ED004BD567
:106D2000294D6E6B26436E639E08284DB60075197B
:106D3000AC46AD689E07360F0F27B740BD43052709
:106D40003F07B84201D1002715E0214FB84201D1D9
:106D5000012710E01F4FB84202D102270BE02BE0C1
:106D60001D4FB84201D1032705E01C4FB84201D1A5
:106D7000052700E00627B7402F436546AF60184D52
:106D80002E684F689643FF0300D516432E606E6849
:106D90004F689643BF0300D516436E60AE684F68D8
:106DA0009643FF0200D51643AE60EE684F689643E7
:106DB000BF0200D51643EE605B1C0A681546DA4038
:106DC00000D057E7FCBD0000001002400000014069
:106DD0000004005000080050000C0050001C00503F
:106DE000000401400069084000D00120704742695A
:106DF00013460B401B0491430B4383617047002AE9
:106E000001D081617047816270470000014880684D
:106E100070470000580100200248816802788918F4
:106E2000816070475801002010B5084800240168AF
:106E3000402211430160204600F00AF8002801D0EA
:106E4000012401E000F042FA204610BD002002407B
:106E500070B504460D4D7D202978C000FEF748F935
:106E600001460B480068FEF743F900F02BFF0028AD
:106E700009D1042C07D200222146401E00F04EFA10
:106E800000206C6070BD012070BD00005801002022
:106E90006401002070477047F8B502F085FE604C31
:106EA0000120E070208AFEF7F0FB01467F20C0053C
:106EB000FEF7EEF95B4D06462968FEF790F928606B
:106EC0000120A16AC005814201DA084603E030468C
:106ED000FEF7DAF9A062FF21C9050025C84200D3F8
:106EE000A562607800280BD102214F48FFF77AFF96
:106EF00002004E494E4817D00022FFF780FFE5629E
:106F000002214948FFF76EFF4A4E002855D0E5623E
:106F1000B08AFEF7BAFB434F3968FEF78DFC5FD2AB
:106F20004549012008705DE00122D1034048FFF788
:106F300066FF208AFEF7A9FB01467F20C005FEF709
:106F4000A7F9E16AFEF74BF93C49E0628842D7DDD8
:106F500038480127F926403000900A213046FEF7D4
:106F6000C7F8002903D131493148FFF701F902215F
:106F70002D48FFF737FF002801D0002701E0002F40
:106F800012D102212848FFF72DFF00280CD104F070
:106F9000CFFD00990120888005F026FB642003F0D6
:106FA00041FE28492648C8600A2003F03BFE3046CF
:106FB000761EF6B20028D0D1A2E7208AFEF765FB44
:106FC00001467F20C005FEF763F9E16AFEF707F985
:106FD0001D49E06288429BDB1A491948C86097E75F
:106FE00015480570708F401EFEF744FB3968FEF7A8
:106FF00023FC06D82079002803D01449012008700A
:1070000001E012480570708FFEF73FFB3968FEF70C
:1070100013FC04D22079002801D004F04BFDF8BD08
:107020001C010020540100200004005000800000DA
:1070300000000050C80D00207600002000004040F5
:107040000400FA0500ED00E00000A04087000020E9
:10705000704770B5040010D0022025462035A87373
:10706000204601F043FDA87B032805D0204600F010
:10707000B9F80020A873687370BD012070BD704717
:10708000704710B5044600680168C943C90708D1B4
:107090008168C943C90704D1012141602046FFF737
:1070A000FBFE20680168C943890708D48168C94389
:1070B000890704D4022141602046FFF7EBFE2068D7
:1070C0000168C943490708D48168C943490704D402
:1070D00004214160204600F0F7F820680168C943A8
:1070E000090708D48168C943090704D4082141600D
:1070F0002046FFF7ADFF20680168C943C90608D4E0
:107100008168C943C90604D4102141602046FFF7B5
:10711000C2FE20680168C943890608D48168C94352
:10712000890604D4202141602046FFF7A9FF20688A
:107130000168C943490608D48168C943490604D493
:10714000402141602046FFF79AFF10BDF8B50400CA
:1071500005D025462035A87B002802D006E0012076
:10716000F8BD00206873204600F04EF80220A87396
:107170002068C26884466368012B01D106208243DF
:1071800016486169814202D0072040038243002BE8
:1071900001D1D82082431248A668024018463043E5
:1071A000676A266A3E433043A66A30431043002B89
:1071B00002D0012B04D005E02369E2691A4300E004
:1071C000E2681043054A914202D0A2691143084384
:1071D0006146C8600120A8730020F8BDFFFF0000D1
:1071E000F8F119FF10B500680549884207D1054834
:1071F000816B4900490881630D2000F073F810BDD0
:10720000007C00400010024010B500680849884228
:107210000CD10848816BC204114381630022012113
:107220000D2000F07BF80D2000F06CF810BD000080
:10723000007C0040001002400068C06970470000F8
:10724000F8B504460220254620351746A8731D4888
:107250000268C3041A4302602068C2689B121A4382
:10726000C260206802690126324302612268102050
:107270005060206881611021204601F0A7FC03289E
:107280001FD02168082048602068476108212046F7
:1072900001F09CFC032814D0204601F027FCA87BB9
:1072A00003280ED02068816831438160206801691D
:1072B0003143016120680169042211430161AE7309
:1072C0000020F8BD00040140704700000448416BF5
:1072D000012211434163816B0204114381637047B2
:1072E00000100240002809DBC106C90E01208840B9
:1072F00003490860BFF34F8FBFF36F8F70470000E3
:1073000080E100E0002805DBC106C90E01208840AD
:10731000014908607047000000E100E010B503F08B
:107320007FFA10BD02494A6882434A6070470000F4
:1073300000700040024801688215114301607047E7
:107340000070004002494A6802434A6070470000EA
:1073500000700040054801680222114301600448A2
:10736000016904221143016130BF70470070004081
:1073700000ED00E0F0B5154A1368154D54152D6A5F
:107380002340ED07ED0F002B04D0002D02D016682E
:10739000A64316601668B608B600064316600D4888
:1073A000076904263743076101290DD040BF20BF7C
:1073B00020BF0169B1430161002B04D0002D02D030
:1073C000106820431060F0BD30BFF2E7007000404D
:1073D0000000014000ED00E0F8B504460078002709
:1073E000534D800671D5524E403EB06BC00004D460
:1073F000B06BA9050843B06301274E480168C90571
:1074000011D40168821511430160FFF7FFFC009061
:1074100005E0FFF7FBFC0099401A642837D845487F
:107420000068C005F5D532680321090560680A4087
:107430000140914208D08103890F032904D13168AA
:10744000890301D50120F8BD2A69032109040A40F6
:1074500022D0084090421FD0207880061CD5286991
:107460002A6988430121C9040A432A612A698A4397
:107470002A612861C0050FD5FFF7C8FC009008E01D
:10748000FFF7C4FC0099411A2B48814201D903201F
:10749000F8BD28698005F3D561688803800F03284B
:1074A00005D132680005824301400A4332602869F1
:1074B000032261681204114008432861002F04D0A0
:1074C000B16B012000078143B1632078C00705D06C
:1074D000E868A168800880000843E8602078800799
:1074E00005D5E8680C218843E1680843E860207806
:1074F000400706D5E86803218902884321690843CB
:10750000E8602078000706D5E8680321090388436E
:1075100061690843E8602078000606D5E868032121
:1075200089048843A1690843E8600020F8BD000091
:10753000401002400070004088130000F8B50E466D
:10754000050038D05E480068C007C00FB04214D2B2
:107550005B4C20684008400030432060FFF756FC39
:10756000074605E0FFF752FCC11B564881427AD816
:107570002068C007C00FB042F4D12878524C800771
:1075800005D5E068F0218843A9680843E0602878C1
:10759000C00752D06868022806D0032807D02168A7
:1075A00001280AD0890504E02168890301E02168E7
:1075B0008901002903DB0120F8BD4907F9E7E168EB
:1075C000890889000143E160FFF720FC07466868ED
:1075D00002280AD0032814D001281ED029E0FFF782
:1075E00015FCC11B374881423DD8E0680007800F79
:1075F0000228F4D121E0FFF709FCC11B3148814288
:1076000031D8E0680007800F0328F4D115E0FFF7B8
:10761000FDFBC11B2B48814225D8E0680007800F85
:107620000128F4D109E0FFF7F1FBC11B2548814295
:1076300019D8E0680007800FF5D121480168C90713
:10764000C90FB14217D901684908490031430160A7
:10765000FFF7DCFB074608E005E0FFF7D7FBC11B9F
:107660001848814201D90320F8BD15480068C007B9
:10767000C00FB042F1D12878400706D5E068072155
:1076800009028843E9680843E0602878000707D5C5
:10769000E0680721C90288432969C9000843E060FE
:1076A00000F03AF8E168094A0906090F515CC84040
:1076B0000749086007480068FFF7CAFBF8BD0000EB
:1076C000002002408813000000100240C2C70008DA
:1076D000640100205C010020044805490068C96875
:1076E000044A4905490F515CC840704764010020B5
:1076F00000100240DBC70008044805490068C9685B
:10770000044A8904490F515CC84070476401002055
:1077100000100240DBC7000870B51A4AD3681A4946
:107720000C2018408D0004280CD04E00082810D0E2
:107730000C2810D050680004410F0120C003491CE0
:10774000884070BD1068C00601D5084670BD284647
:1077500070BD304670BD98020C4C000F205C1B02BF
:107760009C0FD368641CDB0301D5314603E012682B
:10777000D20600D4294603F018F822460023FDF76C
:10778000CDFC70BD0010024000093D00D2C70008CA
:10779000FEB505007ED0FE4CE7680C20E668074089
:1077A0000120000406402878C00747D0082F05D0E4
:1077B0000C2F0AD101200004864206D120688003E4
:1077C0003CD568680028E5D038E0012069680004ED
:1077D000814203D121680143216011E00523012288
:1077E0001B0492049942216802D111432160F1E700
:1077F000814321602168014000912068904320600E
:10780000686800280DD0FFF701FB009005E0FFF746
:10781000FDFA0099401A64287BD820688003F6D5C9
:107820000CE0FFF7F3FA009005E0FFF7EFFA00999C
:10783000401A6428F0D820688003F6D4287880079E
:1078400056D50923E868042F0DD00C2F01D1002E46
:1078500009D000283CD02168994301432160FFF7FB
:10786000D5FA064628E02168490701D5002891D0BD
:1078700061681F22120291432A691202114361605A
:107880002168994301432160FFF746FFE16809063B
:107890000A0F00E08BE1BF49895CC840BE4908601F
:1078A000BE480068FFF7D4FA002873D120E0FFF744
:1078B000ADFA801B0228AFD820684007F7D5606872
:1078C0001F210902884329690902084360600FE00B
:1078D0002068400840002060FFF798FA064604E060
:1078E000FFF794FA801B022896D820684007F7D447
:1078F0002878C00660D5002F0CD0A86900284AD08F
:107900002068FF21013108432060FFF77FFA064617
:107910002EE0C1E02068800502D5A8690028A6D025
:107920006068072149038843296A084360606068EA
:10793000297F0002000A090608436060286A410B9B
:107940000120C003491C8840E16809060A0F9149DB
:10795000895CC8409049086090480068FFF778FA51
:10796000002817D128E0FFF751FA801B0228A2D87F
:1079700020688005F7D56068072149038843296A94
:10798000084360606068297F0002000A0906084316
:10799000606011E0E2E02168FF2001308143216056
:1079A000FFF734FA064604E0FFF730FA801B02289E
:1079B00072D820688005F7D42878794E000724D53E
:1079C00068690028306910D0012108433061FFF751
:1079D0001DFA009005E0FFF719FA0099401A0228F5
:1079E0005AD830698007F6D50FE040084000306172
:1079F000FFF70CFA009005E0FFF708FA0099401A2B
:107A0000022849D830698007F6D42878400766D51F
:107A100000200290A06BC00006D4A06B01210907D2
:107A20000843A063012002905E480168C90511D493
:107A30000168821511430160FFF7E8F9009005E045
:107A4000FFF7E4F90099401A642825D855480068E2
:107A5000C005F5D5FF20AA680130824203D1316903
:107A60000143316111E001218902002A07D0052379
:107A70001B029A4203D132690A433261EFE732694D
:107A800082433261306988433061A868002810D091
:107A9000FFF7BCF9009008E05FE0FFF7B7F9014697
:107AA0000098091A4048814257D830698005F4D5BA
:107AB0000DE0FFF7ABF9009006E0FFF7A7F900999A
:107AC000411A3948814248D830698005F5D4029876
:107AD000002804D0A06B012109078843A063686ACD
:107AE000002866D00C2F3ED00126360602282068DA
:107AF00005D0B0432060FFF789F905462FE0B04379
:107B00002060FFF783F9074604E0FFF77FF9C01B09
:107B1000022822D820688001F7D4E96AA86AE268BE
:107B20000843296BFD231B049A4311430843E0607B
:107B3000206830432060FFF769F9054604E0FFF74D
:107B400065F9401B022808D820688001F7D530E08D
:107B5000FFF75CF9401B022801D90320FEBD206815
:107B60008001F5D425E00128F8D0E068012109045E
:107B7000AA6A014091421AD10F218904EA6A0140A0
:107B8000914214D1032189050840296B88420DE0F8
:107B900000100240C2C70008640100205C01002000
:107BA00040100240007000408813000001D0012006
:107BB000FEBD0020FEBDF8B504000ED0FF27606AB0
:107BC0000537002500280AD0256165612646403624
:107BD000A562707C002807D00AE00120F8BD60682B
:107BE000B842F3D0E561F1E73574204600F03EF885
:107BF000022171742068026840239A4302602123A5
:107C0000A26860689B021A4038401043E3688A0209
:107C10001340184323690B40217D1843C907C90F3E
:107C20000843A169931019400843E16938231940BA
:107C30000843216A802319400843A16A9300194030
:107C4000084321680860A0690421000C0840616AAB
:107C5000102319400843216848602068C169914396
:107C6000C1616565012070740020F8BD10B586B053
:107C7000044614216846FDF79AFA104920688842A4
:107C800019D10F48416B821411434163C16A01222B
:107C90001143C162C06A002110400590E0200090AD
:107CA000022001900320039002910491052069466F
:107CB0000007FEF7DBFF06B010BD000000300140FA
:107CC00000100240094910B5401E884201D9012028
:107CD00010BD074C60610321081F02F0A1FD0020C8
:107CE000A06107202061002010BD0000FFFFFF0001
:107CF00000E000E0F0B502462032137E012B1ED0DA
:107D0000012515760223537606687468B3687027D8
:107D1000BC430F68274377600068AC07A04205D0DA
:107D2000084CA04202D0084CA04204D180244968EB
:107D3000A34319438160557600201076F0BD0220E0
:107D4000F0BD0000000801400014014070B50500BE
:107D500005D02C462034607E002802D006E00120A9
:107D600070BD00202076284600F010F802206076D2
:107D7000291D286801F08EFF0120A077A076E0760B
:107D8000207760776076002070BD000000680121D8
:107D90008907884204D10348816B01221143816322
:107DA0007047000000100240F8B505460446203533
:107DB000287E012817D001262E76022068762268B8
:107DC00090687727FF23B8431B02984390600A68A6
:107DD000502A31D00EDC202A4BD006DC002A48D0B5
:107DE000102A3AD145E00220F8BD302A41D0402A7D
:107DF00033D136E0602A27D0702A12D00120000348
:107E0000121A2AD0824228D1CB684A688968206831
:107E100001F079FF2068816801229203114381609B
:107E20001BE0CB684A688968206801F06CFF216814
:107E300088683843886010E0CA684968206801F0A3
:107E4000DCFF5021206806E0CA684968206801F01C
:107E5000E5FF6021206801F061FF6E760020287642
:107E6000F8BDCA684968206801F0C7FF4021206852
:107E7000F1E711462068EEE710B586B004461421FC
:107E80006846FDF794F9012120688907884212D1DC
:107E90000A49CA6A02200243CA62C96A01900140C3
:107EA00005914102009100210291039104906946DD
:107EB0000348FEF7DBFE06B010BD000000100240D4
:107EC00000040050F8B5064604462036307E0D46C4
:107ED00001280BD0012008273076002A08D0042A78
:107EE00016D0082A2AD00C2A4DD137E00220F8BD3E
:107EF000206801F01BFF2068816939438161206897
:107F0000816904229143816120688169EA6812E0F5
:107F1000206801F023FF206881690122D202114309
:107F2000816120688269012189028A438261206817
:107F30008169EA6812021143816124E0206801F03E
:107F400026FF2068C1693943C1612068C1690422E4
:107F50009143C1612068C169EA6812E0206801F0BC
:107F600031FF2068C1690122D2021143C16120683A
:107F7000C269012189028A43C2612068C169EA6835
:107F800012021143C16100203076F8BD70B50500C2
:107F900005D02C462034607E002802D006E0012067
:107FA00070BD00202076284600F00FF80220607691
:107FB000291D286801F06EFE0120A077A076E076EA
:107FC000207760776076002070BD704770B50546F9
:107FD0002C4602202034002908D004290BD008297F
:107FE0000ED0627F012A10D0012070BDA27E012A2E
:107FF000FAD1A0760AE0E27E012AF5D1E07605E02A
:10800000227F012AF0D1207700E0607701222868E2
:1080100001F06CFE0122286892070121904205D0F0
:10802000074A904202D0074A904204D18268520720
:10803000520F062A02D002680A430260002070BD77
:10804000000801400014014070B504460D46006868
:10805000002201F04BFE2068016A0C4A114203D154
:10806000016849084900016001202034002D06D034
:10807000042D06D0082D06D06077002070BDA076B4
:10808000FBE7E076F9E72077F7E700001111000041
:108090007047704770470000F8B502680446D06921
:1080A00011689668814B05461D402023002D6CD039
:1080B000F7077F4DFF0FBC460D402F4379D0254673
:1080C000C7078035002F06D0CF0504D501271762DA
:1080D0002A683A432A60820708D5F20706D0276843
:1080E00002223A622A6804273A432A60420708D5E6
:1080F000F20706D02668042232622A68022632433A
:108100002A6002070AD50A461A406646324305D05D
:108110002668082232622E6816432E60020508D5B2
:108120004A0106D501222668D20232622A681A4321
:108130002A602A68002A30D0800606D5880604D531
:10814000616E002901D02046884728682168896827
:10815000490602D42821084225D0204602F071F8B1
:1081600020688168490619D5826840218A43826067
:10817000206F002812D04F498163206FFEF7DCFB8F
:1081800000280AD0206F816B06E0850611D58D0688
:108190000FD5616E77E020468847F8BD2046FFF78F
:1081A00079FFF8BD05E02046FFF774FF0020286046
:1081B000F7E7256E012D56D1C50654D5CD0652D50B
:1081C0001026166220688168254649064035002938
:1081D0002ADA226F116849680904090CE1D02F8B53
:1081E0008F42DED9698311680968890617D401684E
:1081F000320191430160206881684908490081602B
:1082000020688168402291438160E36700202066F6
:1082100020680168B1430160206FFEF76BFB288B7B
:10822000698B401A81B21AE0298B6A8B891A6A8B92
:1082300089B2002AB5D00029B3D00268FF252135C4
:10824000AA43026020688268520852008260E36795
:1082500000202066606620680268B2430260204603
:10826000FFF716FF9DE7C50208D5750206D5012068
:10827000000510622046FFF70CFF92E7050605D5C2
:108280000D0603D5A16E002985D18AE7400688D561
:10829000480686D5116820464024A14311608367B3
:1082A0000021816600F043F97BE700000F08000021
:1082B0002001000469A1000810B5040003D0A06FDC
:1082C000002802D007E0012010BD002174200155D4
:1082D000204600F027F82420A0672068016849089C
:1082E00049000160204601F0FFFF0128ECD0606AE0
:1082F000002802D0204601F021FE206841680922B2
:10830000D20291434160206881682A2291438160B2
:1083100020680168012211430160204601F074FECB
:1083200010BD0000F0B587B0064614216846FCF782
:108330003EFF2C493068884251D12B48416B0122C5
:10834000920311434163C16A01221143C162C06AB1
:1083500000251040059003204002009002200327D2
:1083600001A9A1C104200490052069460007FEF779
:108370007DFC1F4C1D48A560E56081C48027E56039
:10838000A7602020256160610002A0611848083CB8
:10839000FEF74CFB002801D0FDF7FEFD3467A66216
:1083A000144C1248214614382060032060601020CD
:1083B0000831A1C16561A561E56120462562FEF72E
:1083C00035FB002801D0FDF7E7FDF466002201210E
:1083D0001B20A662FEF7A2FF1B20FEF793FF07B04B
:1083E000F0BD0000003801400010024030000240A3
:1083F000C41700200C18002070B5C36F202B27D1A4
:1084000000290BD0002A09D0012483682403A34249
:1084100006D10369002B03D1CB0701D0012070BD29
:10842000034660331C7D012C12D001241C750023EF
:108430000366084C0368A34207D05C68240204D595
:108440001C680125AD062C431C6002F04DF870BD80
:10845000022070BD0048004070477047FFB50446D9
:10846000806F83B017460D4620285ED1002D0AD0BC
:10847000002F08D0A168C001814207D120690028DF
:1084800004D1E80702D0012007B0F0BD20466030DB
:108490000090007D012848D000980121017500203E
:1084A000802108512120A067FEF7B0FC2646403607
:1084B0000190378277820120A1680003814202D1B6
:1084C0002069002805D02F46002500990020087556
:1084D00011E00027F9E700228021204602F04AF847
:1084E000002815D1002F15D02168387888627F1CAC
:1084F000708A401E7082708A019B00280698009046
:10850000E9D100224021204602F034F8002808D0AA
:108510000320B9E728882168C005C00D8862AD1C1A
:10852000E6E72020A0670020AEE70220ACE7704716
:10853000034D044C04A002F017F9E560FAE70000CF
:108540000400FA0500ED00E0486172644661756C54
:10855000745F48616E646C65722E0D0A0000000045
:1085600000B585B014216846FCF721FE04490220BD
:10857000C8800449488300F053FC05B000BD0000EA
:10858000080E00201C01002010B50524240700223D
:1085900004212046FEF733FC002208212046FEF786
:1085A0002EFC0A2002F045FB012204212046FEF7A2
:1085B00026FC0A2002F03DFB002204212046FEF7A3
:1085C0001EFC10BD10B505242407002204212046FE
:1085D000FEF715FC012208212046FEF710FC0A20B8
:1085E00002F027FB012204212046FEF708FC0A20A6
:1085F00002F01FFB002204212046FEF700FC10BD04
:10860000F8B5002405260746254636070022042132
:108610003046FEF7F4FB0A2002F00BFB0122042196
:108620003046FEF7ECFB6006040E08213046FEF7EC
:10863000D9FB002801D0641CE4B2052002F0F9FA4D
:108640006D1CEDB2082DE1D3002F03D0FFF79CFF86
:108650002046F8BDFFF7B6FFFAE770B505260546D8
:108660003607002204213046FEF7C9FB0024E80942
:1086700001D0012200E0002208213046FEF7BFFBB6
:108680006806050E0A2002F0D4FA012204213046C1
:10869000FEF7B5FB0A2002F0CCFA00220421304696
:1086A000FEF7ADFB0A2002F0C4FA641CE4B2082C09
:1086B000DDD370BD10B50524240701220821204612
:1086C000FEF79DFB012204212046FEF798FB0022C5
:1086D00008212046FEF793FB0A2002F0AAFA0022A6
:1086E00004212046FEF78BFB10BD10B5052424079E
:1086F000002204212046FEF782FB002208212046AA
:10870000FEF77DFB0A2002F094FA012204212046A4
:10871000FEF775FB012208212046FEF770FB0A20B8
:1087200002F087FA10BD70B505252D07002401223F
:1087300008212846FEF763FB062002F07AFA0122A0
:1087400004212846FEF75BFB062002F072FA07E0E0
:10875000641CE4B2FA2C03D9FFF7C7FF012070BDF7
:1087600008212846FEF73EFB0028F1D10022042113
:108770002846FEF744FB002070BD0000F8B501F06C
:1087800075FC01F0A5FC5B480068C069FDF7F4FCCE
:10879000594C5A49A082898F594E0025002931D061
:1087A000A26A730357499A4202DB02220A7000E070
:1087B0000D700A7801218902002A05D0012A0ED005
:1087C000022A10D0032A1DD1608B01282ED0022846
:1087D00018D1484808214038FFF736FC12E0FF2244
:1087E000F5329042F0D2608B01281DD0022804D0CF
:1087F00008E03046FEF703FB04E03E48082140381D
:10880000FFF7E4FBFDF7C2FD20700121C9023046ED
:10881000FEF7E8FA0127FF0300282DD03A4805604B
:10882000A079002804D007E00022E2E70122E0E777
:108830000120A07101F000FF80213046FEF7D2FA3E
:10884000002806D0002208213046FEF7D8FA01227F
:1088500005E0012208213046FEF7D1FA002205206A
:1088600039460007FEF7CBFA244C284E4034A08C42
:10887000274F012803D01CE0A5710022EAE7254814
:108880006946088072B680212348FDF79DFB0028C9
:1088900004D0022269462048FDF73AFC62B61FA0C8
:1088A00001F062FFA58403F09FFE642002F0BAF994
:1088B000FE60608C012808D110486584058003F0B3
:1088C00093FE642002F0AEF9FE60208C012806D1F0
:1088D000258403F089FE642002F0A4F9FE600748B5
:1088E000124A0188914202D1C088002800D1FE605E
:1088F000F8BD0000401700201C010020C80D00201A
:108900000004005085000020540100200400FA05F6
:1089100000ED00E0AAAA0000384A0008BDF8C8EB44
:10892000C9FDBCB6C4A3CABD0D0A0000AA5500000B
:1089300038B500246946202000F0AAF8684600787F
:10894000572800D001246946212000F0A1F868468C
:108950000078032800D001246946222000F098F80E
:1089600068460078402800D001246946232000F0A2
:108970008FF868460078082800D001246946302026
:1089800000F086F868460078AA2800D001246946DD
:10899000322000F07DF80C486946008F0978884243
:1089A00000D001246946332000F072F80648694679
:1089B000403040880978884201D1002C02D0044917
:1089C0000248C86038BD0000C80D00200400FA0548
:1089D00000ED00E038B55721202000F07AF803219F
:1089E000212000F076F84021222000F072F80821C2
:1089F000232000F06EF8AA21302000F06AF8104819
:108A0000018F142901D8002901D1012101870C4CC3
:108A100040346188142901D8002901D102216180E4
:108A2000008FC1B2322000F054F8A178332000F05A
:108A300050F8684600F006F80A2002F0FAF838BD4F
:108A4000C80D002010B501460F2000F021F80028C5
:108A500000D0012010BD10B50446FFF72BFE3220D8
:108A6000FFF7FBFDFFF75FFEE0B2FFF7F6FDFFF754
:108A70005AFEFFF71FFE3320FFF7EFFDFFF753FE0F
:108A80000020FFF7BDFD0446FFF72FFE204610BD76
:108A900010B50C46FFF7DFFF2070012010BD70B548
:108AA0000D460446FFF706FE3220FFF7D6FDFFF71E
:108AB0003AFEE0B2FFF7D1FDFFF735FE2846FFF79B
:108AC000CCFDFFF730FEFFF710FE0A2002F0B1F8F0
:108AD00070BD10B5FFF7E3FF012010BD10B50248CF
:108AE000FEF7CFFA10BD000078160020FEB5044650
:108AF000002772B6334A01688B1804D13248C76820
:108B000003208004074088680190C8680090486985
:108B10008E69002B08D12C4940398B6ACD042B4338
:108B20008B628B6AAB438B62014631433CD0254953
:108B30002368CB4205D12449CA6803239B049A4386
:108B4000CA6025462035002810D021680A69012313
:108B50001A430A61216848610821204600F036F86E
:108B6000032800D1A873216808204860002E10D087
:108B7000206801690122114301612068866110218A
:108B8000204600F023F8032800D1A87321681020A4
:108B900048600C482168C14206D10B48C1680322D5
:108BA000920491433943C160206801694908490032
:108BB000016121680198886021680098C86062B6E8
:108BC000FEBD00000084FFBF4010024070B50646A5
:108BD0000B480D46002409490068FCF789FA7D21FD
:108BE000C90048433168401E00D103240B682A465F
:108BF0009A4301D00028F6D1204670BD204E0000D7
:108C0000640100201CB5002116480091144A01910E
:108C10000260C16312054260816007228263012203
:108C200002610246C16020321170FF235170C233CD
:108C30004362816211730163816104224163426175
:108C4000C161FDF7BDFC08480090801301906946A2
:108C50000448FDF765FC00210248FDF70BFC1CBD34
:108C6000002401401C1600200200000408B508483A
:108C7000016B012211430163006B01211040009040
:108C800000220A20FEF74AFB0A20FEF73BFB08BD44
:108C900000100240F0B587B014216846FCF787FA4F
:108CA0004748C26A04210A43C262C26A0A40059266
:108CB000C16A80263143C162C16A31400591C16AEF
:108CC00001242143C162C16A21400591C16A022584
:108CD0002943C162C06A22462840059005201C2114
:108CE0000007FEF78CF8012236493748FEF787F86F
:108CF000002236493448FEF782F8912105200022EF
:108D000009020007FEF77BF8314801900027052093
:108D10006946029700940007FDF7A8FF0C20009019
:108D20001120019003200390052002976946000757
:108D3000FDF79CFF10206A46039591C20520694605
:108D40000007FDF793FF11200190029769460397F2
:108D500000941D48FDF78AFF1E4801906946009562
:108D600002941948FDF782FFE002009069460197DE
:108D700002951548FDF77AFF1748694691C1694683
:108D800011480397FDF772FF91200002694691C1D7
:108D90000520694600070397FDF768FF69460A4802
:108DA000019700960294FDF761FF00220121052042
:108DB000FEF7B4FA0520FEF7A5FA07B0F0BD0000F3
:108DC00000100240010200000004005008300000C2
:108DD00000001110000021100832000010B50F4CE7
:108DE0000D482060FF20053060600020A060E0603A
:108DF00020616061E0610121206249026062A1613D
:108E0000A0620720E0622046FEF7D5FE20680168D8
:108E100040221143016010BD00300140A81600201F
:108E200010B58AB00024049405940694079408941D
:108E3000012118480994009401940294890703942D
:108E40000160092184604160046113494461C1608B
:108E5000FEF77CFF01200003049004A90D48FEF7F3
:108E6000A3FF0C48FFF792F8089408A90948099451
:108E7000FEF740FF6020009008480190029408220D
:108E8000694603940348FFF71DF80248FEF7F4FF14
:108E90000AB010BD00170020930400005702000024
:108EA00000B585B014216846FCF781F90E480D49DC
:108EB0000160E1214902416000218160C1600161DE
:108EC00081610C22C1614261016230214162012154
:108ED000090381634900C163FFF7EEF901F0A6FBC6
:108EE00005B000BD00380140401700207047000069
:108EF000F0B585B00A2002F0E7FB7D20400102F0CA
:108F0000FDFBFF4C0025A570FE486066A07C2E4648
:108F10000C2801D30B20A07460790A2801D90A20FB
:108F20006071E570607D002804D0032802D0012024
:108F3000A07600E0A576F448F44F00783871F44943
:108F4000A079097840000843E17D89000843A17EAB
:108F500049010843F871206CF870010A3972401C0D
:108F600020646079B87442003846EA491330FCF74F
:108F700005F96079E74982004000C0196231133079
:108F8000121DFCF7FBF86079062142004843C01926
:108F9000E1491730921CFCF7F1F83220205E0028DE
:108FA00003D0DE49098A081860866079D449C00078
:108FB0002231C2190B7C53764B7C937606227A724F
:108FC000D74A1D301278BA72228D3A73CF4A0B7A83
:108FD000133A1375497A51750022CC4902F05EFCB0
:108FE00060790021C0001D3002F06AFCCD48FEF718
:108FF00023F9A08509E0CB48FEF71EF980B2A085D1
:10900000618FFF392D39884208DB618F80B2884239
:10901000F1D30122920389188842ECD8022002F091
:10902000A3FBBA48C571E574E5730120607425742B
:10903000BC48FEF701F9E0850746E5706079FCF76A
:109040003FFBB94AB94BFCF71FFA01F087FD00223C
:10905000B74BFCF767F9FCF779FB0006C10CC819A0
:1090600080B20121C9032086884201D3401A20869C
:10907000B04820652079401C2071AA48FEF7DCF832
:10908000A085A4489E4F7E3840370190C5E1A54891
:10909000FEF7D2F8A0850BE0A248FEF7CDF880B22B
:1090A000A085218E884203D3A34A8918884207D31A
:1090B00000210F2002F088FAA04960640842EBD03A
:1090C000606C411C1FD040047DD58122D20100215B
:1090D0000F2002F0B8FB0021102002F075FA4106C3
:1090E0008C48490E00229638216602F0A3FA00202F
:1090F00002F004FB002002F0B6FA86489638417A66
:109100000729C3D101E001F0ADFB02228C49401DCB
:10911000FCF758F80028B9D102F023FC784A8032D5
:1091200003C202F00BFC764A8032D1609060E07896
:109130007849401CE0709D390A7A68460270497A85
:10914000417000880390618D88427DD16F497D48D0
:109150008C31C98E01806D4969488C31098FC18479
:109160007048FEF769F8A08502F040F964487D2256
:1091700080308168C068D2040023891858410206F3
:10918000080A10434108490000900A0E08025C4991
:1091900080314A61086108460CC85C480A3002F018
:1091A000B5FB60798100594808185549163080315F
:1091B000CB688A6802F0AAFB514880304369026993
:1091C0005248123000E01BE102F0A0FB4F4808219A
:1091D0004172B430C07C0009A07514D04D48022201
:1091E00057499138FBF7EEFF00280CD10120474981
:1091F000E074C871206ECA311638C2B24548227573
:109200009E30FBF7BBFF6079002280003F491C3095
:1092100002F044FB6079002180001C3002F050FB1A
:10922000009802F04AFA012002F09EFA60730221CF
:109230004548FDF7D7FD002823D0002134480170B0
:1092400032498C31488E00E08CE00090B881888EE5
:10925000F881FF31844621310A68E06C824201D0F6
:10926000761CF6B2206508602A4960659639C97C8B
:109270000907090F032900D06175216E1C2902D04E
:1092800016E00121DAE721491D4A8C31C98F918608
:10929000214A019B143A1B889382884207DD0028EB
:1092A00005DD002903D0207E401C207600E02576D5
:1092B00025710120E073009939826146798220741A
:1092C000E08C2249FF30C33080B2E08488420CD960
:1092D00049424018E0841B487D220188D200491C85
:1092E00089B20180914200D3058016487D21008813
:1092F000C9004843E18C4018A06500F0F1FB27E06D
:10930000700000203F420F001C0100203C12002092
:1093100050010020861300203C150020080E00207C
:109320002C01002078160020B81E85EB51B8CE3FE6
:1093300000000840A0860100983A000000D02724D1
:10934000400100204C01002000040050E703000011
:10935000607B00286AD100210F2002F035F9000659
:10936000F9D563E0FCF7F0FE6F4A032111546F4911
:109370004A8EBA81898EF981216E22461C2905D137
:109380006B4B4100CB1801990988598080006649D0
:10939000664B6039009041189B8F0B8062493039D1
:1093A00041184B68D06C834201D0761CF6B24860FD
:1093B0005E4900988C3940185E491630CB688A683F
:1093C00002F0A4FA616EE06C884208DA564A00990D
:1093D000603A5158012902D16066039902915249BD
:1093E000009A603989582246814216DD012914DD30
:1093F000002812DD0398508502201070A5730CE040
:109400004D4A00210F2002F01EFA6079E178401CDD
:10941000814202D0002002F026F9A18D208E8142E7
:1094200000D234E6454A80188142FAD8E07B012810
:1094300001D00220E07301F0D9FF3F4A00210F2044
:1094400002F001FA2079002818D03D490A889100DD
:109450005118814201D201212170002000F0EAF868
:10946000E07C002835D030490C310B78A372487865
:1094700060728A782272022B17D02AE0216D626E08
:10948000323920468A420EDAC1792D4A491CC9B2C6
:10949000C171128852008A42E2D2029941850221AA
:1094A0000170A573DCE7E571DAE710280CD0C82855
:1094B0000FD2244BC91C1818FBF760FE03F094F878
:1094C000642001F0AFFB1EE6C878FCF7DEF81E4909
:1094D0000860022E04D8E17A481CE072032900D902
:1094E000E57200202378A27B657910E00E4E0E4FC6
:1094F0004100923E7A3F765A7F5ABE4205D00B4FCA
:10950000022300220126A6377E52401CC0B2A84288
:10951000ECD32370A273084A002180320F2002F09E
:1095200092F905B0F0BD000018140020C812002008
:109530003C150020F000002000D02724983A0000BD
:109540002C010020C80D002044010020F8B52E4C4D
:109550000546206F2D4A281A411E6067914215D298
:109560001C21615E081AFCF797F8294A294BFBF782
:109570008BFF064636200F46205EFCF78DF83246FC
:109580003B46FBF7CFFEFCF7BDF8E0860020607697
:109590001D481E23C35E028D1F48008884461F4855
:1095A00006881DE06046484380181D4F80B2388011
:1095B000302778436427643078431A4FA066C01977
:1095C00085420BD2C8B2184936220880A06EA25E2E
:1095D000411BC9188918E1662067F8BD491C6176EE
:1095E000617EB142DED3302042431048642110181E
:1095F00048430F4941182167A0663621401B615E30
:10960000C0184018E066F8BD70000020CF070000C9
:109610009A9999999999B93F3A0100202C01002013
:109620004E01002078ECFFFF380100207427000075
:10963000C0BDF0FFFEB5294D2988491C8FB22849CD
:109640002F800E88FCF728F8264A274BFBF71CFFD3
:109650000191009025483146FBF74AFD244CA18F2B
:109660004218B74206D3002028802248019E1018D5
:10967000009D02E01046019E009DFCF721F8334654
:109680002A46FBF74FFEFCF761F82087012580B2E0
:10969000ED03A84201D3401B2087208CFCF710F873
:1096A000154A164BFBF758FF0646208F0F460090D1
:1096B000FCF706F832463B46FBF734FEFCF746F86B
:1096C00080B26087A84201D3401B60870C49009894
:1096D000096848610098A087FEBD0000380100209D
:1096E0002C0100201904560E2D624040E17A000042
:1096F000700000201F050000F853E3A59B843E4046
:109700007816002070470000F8B531492F480860EE
:1097100002F00EFA2F4800F0A3F92F4CE0822D48FA
:10972000801C00F09DF920832A48001D00F098F964
:1097300060832B4829494180014640310979294FEE
:109740000906090E617006D1C7800121C1870A216F
:10975000418700218187244AC18E1170C18F2171F8
:10976000818F6171817AA17085880521656261812F
:10977000C6883046FBF7BCFCA08101462846FBF7B3
:10978000B7FC8800081885B2164825816843FBF7A6
:1097900097FF164A164BFBF7DFFEFBF7D7FFE0817A
:1097A000658231463846FBF7A3FC20820146C8207B
:1097B000FBF79EFCE0830120A083FCF7DDFCA08288
:1097C000E2890C490C48FDF73BFDF8BD59A600089D
:1097D00068000020004F00081C0100203502000036
:1097E000C80D0020E803000018000020F853E3A58E
:1097F0009B843E40FF7F000078160020F8B5754C32
:109800000027754E2771012030807449C8200880D8
:10981000207B401C2073C00706D0208D411E21856F
:10982000022801D2C82020850120C043FFF702FF93
:109830000A2001F049FF7D20400101F05FFF022175
:109840006748FDF7CFFA00283FD000206549800027
:109850000978664D49000843634909780843A872AE
:10986000102068726248C1887D20C000FBF740FC70
:10987000687360485E490078A87328460B308A7880
:109880000270C97841705A49421C20310B7ED37056
:10989000497E11715649D01C22310B7E5371497E8D
:1098A0009171534940310A7C0271497C4171002217
:1098B0002946172001F0F2FF0021172002F000F8DE
:1098C000022001F051FF4C4D03E00120BEE7FEF7FE
:1098D00055FF00210F2001F077FE28426064F6D08A
:1098E000606C411C73D040046FD58122D2010021ED
:1098F0000F2001F0A8FF0021102001F065FE4106B5
:109900003A48490E0022B430216601F093FE374DEB
:10991000B435687A112858D102223849681DFBF7FE
:1099200051FC002851D1E81F027A69460A70407A3A
:109930004870A97A3180C820FBF7DAFB2749304EFE
:109940000880287B208528462838C08E308029460C
:1099500020482839098FC1842A48FDF76DFCA0856D
:10996000E08C2949FF30C33080B2E08488420BD9B3
:1099700049424018E08430882349401C80B20B31B2
:109980003080884200D3378030887D21C900484329
:10999000E18C4018A06500F0A3F868460088608557
:1099A000A87C12496071C731420008460D468330D9
:1099B000FBF7E4FB6079294642001448FBF7DEFB25
:1099C000208DFF2801D001202070F8BDFFE700F0B6
:1099D00049FF0000700000202C0100203A01002007
:1099E0000004005020010020210100203C12002032
:1099F000C80D00201800002000D0272440010020BE
:109A00004C01002078160020E70300009E13002080
:109A100070B586B014216846FBF7C9FB01250F4ECF
:109A2000ED03002229463046FDF7E9F90120002424
:109A3000019002946946009503943046FDF716F9AB
:109A40000320019002946946009503943046FDF787
:109A50000DF9022001F0E6F806B070BD00040050D8
:109A60000088704770470000F8B5044600206A4639
:109A70001080194D55222A70AA226A700322AA70FA
:109A8000661DEE702A716971144A49008918AC711B
:109A90002246E81DFBF772FB002007E029186A4602
:109AA0008978128889186A461180401CB042F5DB1B
:109AB000611DA81CFCF796F801466846018029192B
:109AC0000078C8716846407808722146093102481A
:109AD00000F0D8FBF8BD0000B6150020C80D00202E
:109AE000FEB5FFF733FD2548FDF7A6FB244C86B2F3
:109AF000A68560790A21081AC000FBF7CDFD07464C
:109B00000191E06EFBF7DCFD1E4A1F4BFBF724FDC5
:109B100000900D463046FBF7D3FD2B46009AFBF72D
:109B200001FC3A46019BFBF7FDFBFBF70FFE85B2FC
:109B30002587208CFBF7C4FD124A134BFBF70CFD65
:109B400006460F462846FBF7BBFD32463B46FBF771
:109B5000E9FBFBF7FBFD81B20120C0036187814275
:109B600001D3091A6187854201D3281A2087034946
:109B7000208F09684861A087FEBD0000781600208C
:109B800070000020F853E3A59B843E40034A11680F
:109B9000382389B299430143116070470030014076
:109BA00010B5FDF739F910BD10B59AB034216846EB
:109BB000FBF7FDFA14210DA8FBF7F9FA1C2112A8F6
:109BC000FBF7F5FA1B4801680324E402A143C21421
:109BD00089180160FDF7AEFB17480169A1430161D7
:109BE00006200090FF2001300290012003901020F9
:109BF00004900220099040040B90000100240C9076
:109C00000A946846FDF7C4FD0F200D9003200E90C6
:109C10000F941094012111940DA8FDF78FFC812061
:109C20001290032080041890149412A8FDF7D4FB1E
:109C30001AB010BD0070004040100240104801688A
:109C4000821511430160C1680E4A1140C16001686C
:109C50000D4A11400160816849084900816001682E
:109C60000122920491430160C168FD2212049143D4
:109C7000C160002101610649044888607047000006
:109C8000001002400C40FF88F6FFF6FE005000086E
:109C900000ED00E070B5026801239B07114C124DE6
:109CA000984203D0A04201D0A84203D17026B2430B
:109CB0004E683243984203D0A04201D0A84204D15A
:109CC00003231B029A43CB681A4380239A430B69F0
:109CD0001A4302608A68C262096881620121416197
:109CE00070BD0000000801400014014010B5CB0613
:109CF000DB0E0121046A99408C430462016A9A4098
:109D00001143016210BD30B58468FF252D021B028E
:109D10001343AC430B432343836030BD82687023FD
:109D20009A430A4307210A438260704730B5026AAA
:109D3000520852000262026A456883697024A34394
:109D40009C080B68A40023430224A2438C6845604E
:109D50001443836149684163046230BD30B5026ACF
:109D600010239A430262036A4568826973242402BD
:109D7000A2430C6824021443202293438A6845605E
:109D800012011A43846149688163026230BD30B5B3
:109D9000026AFF2301339A430262026A4568C3697B
:109DA0007024A3439C080B68A4002343012464028D
:109DB000A2438C68456024021443C3614968C163AF
:109DC000046230BD30B5026A01231B039A4302626C
:109DD000036A4568C26973242402A2430C68240202
:109DE00014430122520393438A68456012031A43C5
:109DF000C46149680164026230BD30B5036A046A17
:109E00006408640004628469F025AC4312012243B3
:109E10000A24A3430B438261036230BD30B5036A59
:109E20001024A34303628469036A0F252D031203E0
:109E3000AC432243A024A343090119438261016278
:109E400030BD0000F8B5102405252D07AC62AF2009
:109E5000800000F0EEFEAC6101F0CAFB2D4C2E4FED
:109E60002E4EA0670EE001F0C3FBA067FEF786FC54
:109E7000A06C411CA164142804D929A000F074FC32
:109E80002B48C760A06FB042EDD10026A6642078B1
:109E90000127FF03030000F0A0FC04030B182C2E85
:109EA000012239462846FCF7AAFFFFF7A7FC06E087
:109EB000012239462846FCF7A2FFFBF7C3FE002229
:109EC00039462846FCF79BFF15E0A07B0122401C89
:109ED000A07339462846FCF792FFFCF769F9002287
:109EE00039462846FCF78BFFA07B052803D926704E
:109EF00001E0FEF7FDFF02210E48FCF773FF00288A
:109F000005D000200C49087001F058FAF8BD012076
:109F1000F8E70000700000200400FA053001CADEF6
:109F20004457204944204552524F522E0D0A0000FA
:109F300000ED00E0000400505001002010B5818CBD
:109F4000C90707D001684A6801235B049A43836A02
:109F50001A434A60818C890707D501684A68012342
:109F60001B049A43C36A1A434A60818C490707D588
:109F700001684A6801239B049A43036B1A434A60B1
:109F8000818C090707D501684A680123DB039A43DE
:109F9000436B1A434A60818CC90607D502689168F1
:109FA00001231B039943836B19439160818C8906BC
:109FB00007D501688A6801235B039A43C36B1A4380
:109FC0008A60818C490612D503685A680121090507
:109FD000046C8A4322435A60026C8A4207D10268A9
:109FE000516803235B059943436C19435160818C8D
:109FF000090607D501684A680123DB04806C9A438F
:10A0000002434A6010BD0000F8B5044600268030C7
:10A010000660FCF7FBFE054620680068124F00074B
:10A0200009D501212B46002249052046009700F062
:10A03000A1FA00280DD12068006840070BD5012146
:10A040002B46002289052046009700F093FA00284D
:10A0500001D00320F8BD2020A067E06726666034A9
:10A0600026750020F8BD0000FFFFFF01F8B5154C74
:10A07000C826E078002823D16079002820D101206B
:10A080006071114D686B0027002818D0686BC821DB
:10A09000081A0FE00D48E168405C61698847E06894
:10A0A000401CE060E068C82800DBE760696BC820FE
:10A0B000401A761EE168814201D0002EEADC677109
:10A0C000F8BD00005400002000000240000D0020F8
:10A0D00070B5224CE07800283FD1207900283CD18F
:10A0E000012020711E4EF16900250906002933DA8E
:10A0F0002156625791420AD1F06940062CD5A079C9
:10A10000002829D0A5712089401C208124E0A17954
:10A11000002903D1A0710A2000F08BFD00202056F9
:10A12000CC2148430F494218206912181279B262B3
:10A13000401C00222061A256CC235A4389588142F8
:10A140000ADC25612078401C207020780E2800D180
:10A150002570A078401CA070257170BD54000020AF
:10A1600000380140D801002010B5806A0022014665
:10A1700040314A834A82FDF78DFF10BD70B5846A75
:10A18000A06FE56F2168896800260906002906DAB4
:10A19000212804D152200653204600F06BF8206895
:10A1A0008068400606D5222D04D15A200653204649
:10A1B00000F047F82046803001681022114301600A
:10A1C0002046FDF767FF70BD10B501460968806A3B
:10A1D000096889061CD400225A210A5201680A68BB
:10A1E000FF2301339A430A6001688A6852085200CB
:10A1F0008A6001688A6840239A438A602021C16787
:10A20000016E012904D101680A6810239A430A608B
:10A21000016E012902D0FEF71FF910BD5821095A1D
:10A22000FDF736FF10BD10B5806A016E012902D01E
:10A23000FEF713F910BD5821095A4908FDF728FF08
:10A2400010BD01680A68FF2321339A430A60016840
:10A250008A68520852008A60016E012904D101689F
:10A260000A6810239A430A602021C1670021016611
:10A270004166704701680A68C0239A430A6020213A
:10A280008167704770B5164CE278002A0CD12279AC
:10A29000002A09D10122E2700025C82903DC02222C
:10A2A000A256002A01DCE57070BD0123E356CC22E2
:10A2B00053430C4AD1500123E356CC2673439B18D9
:10A2C0000A460146181DFAF759FF6078401C607075
:10A2D00060780E2800D16570A078401EA070E2E77B
:10A2E00054000020D8010020F8B5044601688068B9
:10A2F0002369E66918436369002533431843724AAA
:10A300000B68724E334003430B6021684868032397
:10A310001B039843E368184348602168A069914291
:10A3200001D0236A18438B680B263602B3430343DC
:10A330008B606749236867488B420CD1C0688007EF
:10A34000800F06D0012839D0022835D0032821D12A
:10A350001EE001271FE060498B420AD1C0680C2132
:10A36000084027D0042829D0082825D00C2811D14E
:10A370000EE093420ED1C16803208002014019D043
:10A3800001208002091A19D0091A15D0814201D181
:10A39000082700E010274F49504840398600934273
:10A3A00032D1002F0CD0022F0DD0042F10D0082F47
:10A3B0007FD126E00027EEE70227ECE70427EAE753
:10A3C000FDF78AF906E00968C90605D4304603E0BE
:10A3D000FDF7A2F9002872D062685100511881423D
:10A3E00067D81103814264D3010E0602500800238E
:10A3F00030185941FAF792FE03210902411A384AEE
:10A4000055E00120C003E7E70122E369D20393424C
:10A410002BD13B0000F0E1F90906090C4D114D4D1F
:10A420004D274D00FDF758F909E0FDF765F906E005
:10A430000968C90605D4304603E0FDF76DF9002828
:10A440003DD0616840004A088018FAF751FE80B29A
:10A450000146244A103991422BD8511C0140000773
:10A46000400F084329E01046EBE73B0000F0B5F948
:10A470000906090C2112212121232100FDF72CF9C5
:10A480000AE0FDF739F907E00968C90606D4304645
:10A4900004E00EE0FDF740F9002810D061684A089A
:10A4A0001018FAF725FE80B201460E4A1039914283
:10A4B00003D9012503E01046F0E72168C8600020B9
:10A4C0006066A0662846F8BD00480040F369FFEFCB
:10A4D00000380140401002400044004000093D00A7
:10A4E000FFFC0F00EFFF0000F8B504464165403067
:10A4F00000262746028380373E602220E0672546FB
:10A50000206F603500281CD01749C162216F1748A1
:10A510000863216F16484863206F8663236F606D60
:10A520009C4613462168024660462431FCF7C6FA71
:10A53000002806D0102038602E752020A06701204A
:10A54000F8BD2E7520680168FF22013211430160B9
:10A55000206881680122114381602068816840225F
:10A56000114381600020F8BDC9A1000827A200089E
:10A570007DA10008FFB581B005460F460446603551
:10A580000A9E39E0701C37D0FCF740FC0499401A51
:10A59000B04222D8002E20D02068016849072BD570
:10A5A000C069C043000527D401202168C0020862A9
:10A5B00020680168FF22A132914301602068816810
:10A5C0004908490081602020A067E067803420604E
:10A5D00000202875032005B0F0BD20680168FF2227
:10A5E000A132914301602068816849084900816077
:10A5F0002020A067E067EBE72068C1693846884300
:10A6000005D0002103988142BCD00020E3E701215E
:10A61000F8E7000010B504491020096808620248F4
:10A62000FDF73AFD10BD00004017002001490D2044
:10A63000887070475400002010B5FEF717FBFEF736
:10A640002FFCC82202490348FDF7D6FE10BD0000CA
:10A65000000D002040170020F8B53E4C0023217863
:10A660003D4A1D46082910D0072947D0062950D059
:10A67000052952D0042953D0032954D0002956D09B
:10A68000012958D002295AD05BE0A17800264A1F40
:10A6900004E0314FBF5DFB189BB2761C9642F8DB9D
:10A6A000667927799A195118E3786278C918891858
:10A6B000C9194018C0430006000E1AD1012E14D04B
:10A6C000022E16D125482449C018FAF757FD01F08B
:10A6D0008BFF642000F0A6FABFF34F8F214920487A
:10A6E000C860BFF34F8F00BFFDE759081046FFF762
:10A6F000BBF92570E570A570A571F8BDA17950541E
:10A70000491CC8B2A071A178491F8842F5D1082020
:10A7100001E0607007202070F8BDE0700620FAE7C5
:10A7200060710520F7E7A070E5700420F3E7552875
:10A7300007D10120EFE7AA2803D10220EBE7032885
:10A7400003D02570E570A570F8BD0320207020713E
:10A75000F8BD00001301002052150020C80D002094
:10A760000400FA0500ED00E010B5024A024900F0CD
:10A77000E5F910BD25B90008680100202021020C70
:10A7800001D010211046020A01D0104608390209F2
:10A7900001D01046091F820801D01046891E4208C8
:10A7A00001D0881E7047081A7047F8B5040C8BB2A8
:10A7B000264682B25E430D0C1046370C58433604D1
:10A7C00080190021794116466E43370C36048019F2
:10A7D000794126466E438919F8BD30B47446641E2B
:10A7E0002578641CAB4200D21D46635D5B00E31814
:10A7F00030BC18474900CA020243100000D00420B0
:10A800004A0D01D001221043044A490D914201D161
:10A8100002210843012800D105207047FF070000EE
:10A820008307FF22DB0E9A408907090E9940002812
:10A8300008DB830809489B001B18186890430843ED
:10A84000186070470007000F0838830804489B0011
:10A850001B18D86990430843D861704700E400E0B2
:10A8600000ED00E0BFF34F8F04490348C860BFF319
:10A870004F8F00BFFDE700000400FA0500ED00E087
:10A88000F8B504464F1EC8000838211815461E4664
:10A89000086849683A4606239A4310D02A46334648
:10A8A000FAF7F2FD3A46D200083AA3181A687F1E5A
:10A8B0005B68FAF737FD06223B469343EED1022F41
:10A8C00023D0042F11D0062F2FD12A463346FAF772
:10A8D000DBFDE36AA26AFAF725FD2A463346FAF75A
:10A8E000D3FD636A226AFAF71DFD2A463346FAF75A
:10A8F000CBFDE369A269FAF715FD2A463346FAF75C
:10A90000C3FD63692269FAF70DFD2A463346FAF75B
:10A91000BBFDE368A268FAF705FD2A463346FAF75D
:10A92000B3FD63682268FAF7FDFCF8BD002210B59C
:10A93000134610460149FAF70FFE10BD0000F03F24
:10A9400010B5FAF7EFFC10BD002210B51346104603
:10A950001146FAF701FE10BD10B50721024A00208A
:10A960000907FAF771FE10BD01030000034A10B594
:10A9700000201107FAF768FE10BD000001FDFFFF7F
:10A9800002E008C8121F08C1002AFAD170477047B8
:10A99000002001E001C1121F002AFBD17047000016
:10A9A00001490860704700006C01002008B50021D3
:10A9B000684601706B46012202212C2000F052FFF4
:10A9C0000221684601706B4601222C2000F04AFFEC
:10A9D00008BD000038B504466D20694608706B4616
:10A9E000012207492E2000F03DFF0649002C01D02E
:10A9F000054A00E0054A2E2000F01AFF38BD00008D
:10AA000006080000061800000706000007160000F0
:10AA100038B504466B4602220021362000F0EEFDD8
:10AA2000B3212300FFF7D9FE0E0F08153A3A3A3A40
:10AA30001C273A3A2F34483A002168460170407882
:10AA40004108490014E06946087880088000401CED
:10AA500004E06946087880088000801C08701DE0CA
:10AA6000684602780A4048320270417880200143EB
:10AA70006846417012E0684602780A4002704078E9
:10AA80004106490EF4E7694648780221084303E08D
:10AA900069464878FD210840694648706B460122A6
:10AAA0000021362000F0DEFE012200AB11463620E8
:10AAB000013300F0D7FE38BD69460878CF21084041
:10AAC00069462030CAE708B5032168464170012174
:10AAD00001706B4602220021362000F0C3FE0122E5
:10AAE000D20306212D2000F0A3FE012000F09AF8E9
:10AAF0000120FFF78DFF08BD08B5020A69464A70BC
:10AB000008706B46022204212D2000F0ABFE0320CA
:10AB1000694608706B46012206212D2000F0A2FE36
:10AB20000020694608706B46012206212D2000F0A6
:10AB300099FE0A212D2000F047FD08BDF8B5164604
:10AB40000F460446002503E03946B047641C6D1CDF
:10AB500020780028F8D12846F8BD0000F8B54A0052
:10AB60002B4B520DD6182B4A0C460546142E2BDAC9
:10AB7000002E12DA284BFAF7D5FB00221346FAF71B
:10AB80002BFE40D2002C03DA0124E40700253AE032
:10AB90002046284337D0214C14E0214F0B46F74084
:10ABA0003B402B4331D01C4BFAF7BCFB0022134631
:10ABB000FAF712FE27D2002C03DD01200005F04039
:10ABC0000419BC4300251EE0332E1EDC334600274B
:10ABD000143BFF43DF40384217D00F4BFAF74CFCD1
:10ABE00000221346FAF7F8FD0DD2002C0ADD142ED0
:10ABF0000CD03420811B012088404019A84200D28B
:10AC0000641C0546BD4321462846F8BD641CF9E78F
:10AC100001FCFFFF9C7500883CE4377E0000F03F9C
:10AC2000FFFF0F007D2110B5C900484300F001F877
:10AC300010BD002140E000BF00BF00BF00BF00BF4B
:10AC400000BF00BF00BF00BF00BF00BF00BF00BF0C
:10AC500000BF00BF00BF00BF00BF00BF00BF00BFFC
:10AC600000BF00BF00BF00BF00BF00BF00BF00BFEC
:10AC700000BF00BF00BF00BF00BF00BF00BF00BFDC
:10AC800000BF00BF00BF00BF00BF00BF00BF00BFCC
:10AC900000BF00BF00BF00BF00BF00BF00BF00BFBC
:10ACA00000BF00BF00BF00BF00BF00BF00BF00BFAC
:10ACB00000BF00BF00BF491C8142BCD37047FFB535
:10ACC00081B01E460F46040026D00B99039801431D
:10ACD000A06A3943826807209047002818DB0A9948
:10ACE000A06A3143826806209047002810DB254681
:10ACF0002035A979032F01D908200143032E01D95A
:10AD000004200143A06A826809209047002806DADF
:10AD10000120C04305B0F0BD0020C043FAE738462B
:10AD200000F000F92060304600F0FCF860600A98FE
:10AD300068700398A870EF702E710B9868710020EE
:10AD4000E8E70000F7B50446002090B000900190BD
:10AD5000002C05D06A46062101F080FC062803DAA3
:10AD60000020C04313B0F0BD684640780102684639
:10AD7000007800040918684680780818FAF7A0FCE3
:10AD8000054668460391007901026846C0780004D0
:10AD90000918684640790818FAF792FC032206461B
:10ADA0000F4692075C4BFAF717FD07D200225B4B68
:10ADB00030463946FAF75AFB06460F4603229207F9
:10ADC000554B28460399FAF707FD07D20022534B4B
:10ADD00028460399FAF74AFB054603912068FAF7DB
:10ADE0006FFC02460B4630463946FAF7B5FB07467C
:10ADF0000A200791205EFAF74FFC3A46079BFAF7C4
:10AE000043FB064608200991205EFAF733FC002137
:10AE1000C943FAF77BFAFAF7B7FC3246099BFAF70F
:10AE200081FA069108906068FAF74AFC02460B46E0
:10AE300028460399FAF790FB05461A200E46205E35
:10AE4000FAF72AFC2A463346FAF71EFB0C900991C2
:10AE50001620205EFAF720FC099B0C9AFAF762FA9A
:10AE600005910A902A46334638460799FAF70CFBB3
:10AE7000059B0A9AFAF708FB05910A901420205EB8
:10AE8000FAF70AFC3A46079BFAF7FEFA07461C2037
:10AE90000791205EFAF700FC2A463346FAF7F4FAE7
:10AEA0000E900B911820205EFAF7F6FB0B9B0E9A82
:10AEB000FAF738FA2A463346FAF7E6FA0B910E907B
:10AEC0002069FAF7E9FB0B9B0E9AFAF72BFA2A4650
:10AED0003346FAF7D9FA05460E46E068FAF7DCFB86
:10AEE0002A463346FAF71EFA3A46079BFAF71AFA49
:10AEF000059B0A9AFAF716FA01229207084BFAF70D
:10AF0000C3FA02460B46129C0898069903C411988E
:10AF10000CC0002026E70000FFFF5F4100007041E9
:10AF2000E17A843F00B50121C9040300FFF755FC15
:10AF3000081A05080B0E1114171A0320C00400BDCF
:10AF40000720C00400BD0F20C00400BD1F20400327
:10AF500000BD3F20400300BD7F20400300BDFF2017
:10AF6000400300BD084600BDFEB5264F0D46040057
:10AF70000FD0002D0DD0264600202036B071F07184
:10AF800029680D208847002801DA7800FEBD1028C6
:10AF900001D03846FEBDA562E968002901D028200D
:10AFA0008847204600F030F80028F3DBA06AA5218E
:10AFB00082680E209047A06A962182680F209047F1
:10AFC000A06A0221826862209047A06A00218268FC
:10AFD0000E209047A06A002182680F209047717967
:10AFE0003020019100900623202201212046FFF706
:10AFF00066FE0028CEDB204600F0AEF80028C9DB54
:10B000000020FEBDFFFFFFFF10B586B004461421EF
:10B010006846FAF7CCF8002C7ED0A06A122143686B
:10B020006A4610209847122877D168460078012296
:10B03000010168464078120300090818434920813D
:10B04000884201DD801A20816846837840780007B5
:10B05000000D18186081884201DD801A6081684601
:10B060000079012201016846C07812050003091821
:10B0700068464079000908183549E060884201DDDA
:10B08000801AE060684640790007030B68468079C3
:10B0900000021B186846C07918182061884201DD3B
:10B0A000801A20616846417A007A0002081802B2CC
:10B0B000284801210904A282824201DD521AA2829B
:10B0C0006A46D37A927A12029A1812B2E2828242C5
:10B0D00001DD521AE2826A46537B127B12029A18F1
:10B0E00012B22283824201DD521A22836A46D37B46
:10B0F000927B12029A1812B26283824201DD521AC6
:10B1000062836A46537C127C12029A1812B2A2839E
:10B11000824204DD501A01E00BE008E0A083A06A3F
:10B12000016828208847002806DA0120C04306B0BD
:10B1300010BD0020C043FAE7C011C007203400282A
:10B1400000D0802060710020F1E70000FF070000C0
:10B15000FFFF0700FF7F000010B5040009D0A06AC0
:10B160000721826808209047002805DA0120C043A3
:10B1700010BD0020C04310BD0720203420700020E7
:10B1800010BD0000FEB504460020019000906079DB
:10B19000734940000E5A61782578491E7148CFB234
:10B1A0000163042D77D0072D75D0002102912178FD
:10B1B00001736C49E379012292058969002B6CD0F7
:10B1C000914381616748217A4173217A82698907B5
:10B1D000890B0A4382610021042000F034FB3246CF
:10B1E00061492E2000F024FB3846FFF7F3FB5F4E49
:10B1F0000522705D810040185D49431807212B200E
:10B2000000F030FB5B49029801220B180B2128202B
:10B2100000F028FB705D584980000A580C21282056
:10B2200000F011FBE079554980004018A1794900F0
:10B23000425A0221272000F0FBFA51487E00825B2F
:10B240000421272000F0F4FAE079002829D0A07822
:10B2500004282CD0282069460872202206212720A5
:10B2600000F0E6FA02AB01222621272000F0FAFACC
:10B27000444938014018E1788900425808212720C4
:10B2800000F0E1FAA17A601C627A0902114313D03E
:10B2900016E000E001E0012188E71143F608816132
:10B2A00090E764220621272000F0C2FAE0E7102090
:10B2B000694608720246D1E733490172090A4172B0
:10B2C000417A007A0A0202432021272000F0B0FAD6
:10B2D0002E4F0C2123203A6800F0B5FAF01982882D
:10B2E0000421232000F0A4FAA07900280BD0E079F3
:10B2F0002749012243180021212000F0B3FA03203E
:10B300000190012000902A07120F1001024360787B
:10B3100000218007000B02430198000502430098BA
:10B32000400402432079C006400902436079C00608
:10B3300002431F2000F087FAA078617801230843B8
:10B3400002040848DB030261E179490319430A4317
:10B3500002610021082000F076FA0020FEBD000006
:10B3600090C700089C0100200428000038C700088E
:10B37000240000204200002040C7000860C70008E9
:10B380006CC7000870C700084110000058C70008CB
:10B390004400002038B50C4607498A8B002102433F
:10B3A0002C2000F045FA684604706B460122062105
:10B3B0002C2000F057FA38BD9C01002010B5FFF793
:10B3C000F5FA10BD10B504460421362000F0FCF853
:10B3D0000121C902002C01D0084300E08843024645
:10B3E0000421362000F02FFA10BD000038B54020AF
:10B3F0006946087000210E2000F0E6F8044600229D
:10B4000011460E2000F01FFA6B46012200210D208C
:10B4100000F028FA074A00210F2000F014FA00F08B
:10B42000EDF9224600210E2000F00DFA024800211D
:10B43000017338BDF8FF2724BC010020FEB5054686
:10B44000042069460870514C002060752146203167
:10B45000206348710873A0836063A06300F0C8F89C
:10B460004B4E206002E000F0C3F82060B042FAD1F9
:10B470000020FFF7CDFA00F0BBF8464E2060307890
:10B48000242801D9243806E00621F9F731FE0622E6
:10B49000101A40010843020601040A4301020A434C
:10B4A0000243B260706000211E2000F0CCF900F071
:10B4B0009FF820606B4601220021242000F0D2F981
:10B4C0001E20FFF719FB86B2300AA0730420FFF795
:10B4D00013FB074600F08CF820603806000E0DD0F4
:10B4E00002206946087101AB012212212D2000F0D3
:10B4F000B9F9A08B012109030843A08300F078F873
:10B5000020600620FFF7F8FA60600720FFF7F4FAE2
:10B51000A060F006C00E207501D110202075C0B2C9
:10B5200000F0DCF9E80707D0FFF7CDFAA08B012186
:10B53000C9020843A0830AE00521362000F02EF856
:10B540001549084002460521362000F071F9012016
:10B55000FFF75EFA0021042000F036F8A061002118
:10B56000262000F031F81521890308430246002106
:10B57000262000F068F900222621362000F058F934
:10B5800000F036F820600020FEBD00009C01002085
:10B590003001CADE18000020FFFD000038B5094C5C
:10B5A00089B280B26B46022200F028F8002806D14A
:10B5B00068464078010268460078081884B2204640
:10B5C00038BD0000FFFF000038B50024E44389B215
:10B5D00080B26B46042200F011F8002806D1032146
:10B5E0006846435C2202D418491EFAD5204638BD6D
:10B5F00010B500210846FFF7E7FF10BD38B5002958
:10B6000009D0402420436C462070C8B27F2906D858
:10B61000607002200AE069460870012006E080247C
:10B6200020436C466070C809A0700320694600F092
:10B63000B5FF38BD10B5144603460A462146112011
:10B64000FFF7DCFF10BD10B50346052200211520D1
:10B65000FFF7D4FF10BD10B50346052200211720C7
:10B66000FFF7CCFF10BD38B50546002069460870CD
:10B6700000F0C4F8FF2401342246002D01D003223B
:10B68000120200210D2000F0D3F8002D13D06B46DC
:10B69000012203210F20FFF7B1FF68460078000761
:10B6A00009D5FFF7A3FE224600210D2000F0C0F8C7
:10B6B0000020C04338BD002038BD10B5024601212E
:10B6C0000A2000F0C0F810BD10B5044600211A2071
:10B6D000FFF77AFF000D22030005120B0243002141
:10B6E0001A2000F0B0F810BD10B5024602492E2015
:10B6F00000F09EF810BD000004180000F8B50546E3
:10B700006B46012203210420FFF778FF0126114C2C
:10B710003607002D0DD02A4600210C2000F088F8B5
:10B72000694608781021084369460870A0693043CB
:10B7300007E069460878EF21084069460870A0696B
:10B74000B0430B46A06101220321042000F08AF8D7
:10B75000F8BD00009C01002010B502460021182011
:10B7600000F066F810BD0000F8B5074600256846F1
:10B770000570B807204C2E4600280ADA802069465A
:10B7800008706B46012200210D2000F06BF80120AB
:10B790002073F8076946087821D0062108436946D6
:10B7A00008706B46012200210D2000F05BF8032198
:10B7B0000F20FFF7F3FE8121C900084219D0402075
:10B7C000694608706B46012200210D2000F04AF8FE
:10B7D0000020FFF7F7FD00252673ED4309E0022165
:10B7E0000843694608706B46012200210D2000F0D5
:10B7F00039F82846F8BD0000BC0100201CB56B4696
:10B80000012203210F20FFF7F9FE6846007840224D
:10B81000C1091040C9014000814208D00120694699
:10B820000871024601AB03210D2000F01BF81CBD7E
:10B8300008B56B461A70120A5A7089B280B2022299
:10B8400000F010F808BD38B500236C46E254120A27
:10B850005B1C042BFADB89B280B22346042200F081
:10B8600001F838BD38B58024002909D0C025284307
:10B870006D462870C8B27F2907D86870022009E099
:10B88000204369460870012004E020436870C8091D
:10B89000A8700320694600F02BFF38BD10B5144690
:10B8A000012312189B029A4202D90020C04310BD06
:10B8B0000B46821E21460920FFF7D4FF002010BD51
:10B8C00010B5054A8905126901430A430021082081
:10B8D000FFF7B9FF002010BD9C01002038B50446D9
:10B8E0006B4601220E212B20FFF788FE6846007868
:10B8F000E10640094001C90E0143684601706B46EC
:10B9000001220E212B20FFF7ADFF38BD10B500211D
:10B9100042541C06120A22431B0A491C0429F7DB65
:10B9200010BD000013B501231A4669460248FCF712
:10B9300095FD00981CBD0000401700207CB5002438
:10B9400025466846FFF77FFE04206946220E2D0239
:10B95000154322020C5C1443401EF7D520462946AD
:10B960007CBD7CB5002425466846FFF774FE0420A4
:10B970006946220E2D02154322020C5C1443401E20
:10B98000F7D5204629467CBDFBF74EFAFEF70CF9A9
:10B99000FDF780F93F494048002522C005608561D8
:10B9A000C5613E490562C1600838FBF7CFFBFDF772
:10B9B0005DF9FDF775FAFDF711FAFDF723F9052496
:10B9C00001222407D1032046FBF719FAFDF79CFE5C
:10B9D000FDF700F8FAF7E2F8FAF78CFAFAF75AFAF4
:10B9E000FCF7BEFD0721A015FFF7D4FCFFF7E6FC2E
:10B9F000012211032046FBF702FA2748C8222849F2
:10BA0000C830FCF7F9FCFCF793FF264F264E274C75
:10BA1000387800280FD13078002801D003280AD1C7
:10BA20000121C9022248FBF7DDF9002803D10121D9
:10BA30000846FBF79FFCE078002828D060780028B3
:10BA400025D0E57072B620780F280AD90120184950
:10BA500000038861FEF7F6F90120154900038862AA
:10BA60000CE0012251031248FBF7C9F9FEF7EAF98D
:10BA70000121002249030E48FBF7C1F962B6FCF729
:10BA80007DFE208C0028C3D0401E2084C0E7FCF738
:10BA900075FEBDE7007C004078160020FFFF000027
:10BAA000000D00205A000020850000201C0100200D
:10BAB0000004005010B586B01848FBF7CAFA1421EC
:10BAC0006846F9F774FB16480090032001900020A7
:10BAD0000290052069460007FBF7C8F8694611483F
:10BAE000FBF7C4F869461048FBF7C0F8FCF720FFE5
:10BAF00001210846FBF73EFCFF2401342046FBF7FA
:10BB000011FC0A4908680422104308602046FBF72C
:10BB100019FCFBF71FFC06B010BD000078160020D2
:10BB2000FFFF0000000400500008005000700040BB
:10BB300010B50122920217491748FAF75FFA154823
:10BB4000164902888A4223D0018004218180FF2186
:10BB5000F531C1800A21018100211E224181D24399
:10BB600082810122C28181834323C386022303870A
:10BB7000782343878287C2870246403211845184EA
:10BB80009184C183918014238382118200F02CFD63
:10BB900010BD0000C80D002000FC0008AA550000E0
:10BBA000F0B51FB496B084460C460246199D18980D
:10BBB0000390490068006300490840080193002A87
:10BBC00001D0012600E000269E19FE4BF6185B10FE
:10BBD0009E422BD36E00039F0296002F00D00127B8
:10BBE000F719F84EF84BBE199E421FD3039E034629
:10BBF000F64F334309D03B469C4201D1002A04D082
:10BC0000019B002A05D0012604E0002039461BB024
:10BC1000F0BD00269E19EE4B9E4207D8039F029E60
:10BC2000002F00D00127F6199E4207D92B46604607
:10BC30002146189AFEF784FE1BB0F0BD0023002CAD
:10BC400029DAE44EB04226DAE34EB04201DB0223A9
:10BC500021E0DE4EB0421EDBE04E070DBE19142E71
:10BC600009DD3427BF1B039EFE400196BE40039FA3
:10BC7000BE420BD00FE0039F002F0CD11427BF1B37
:10BC80000646FE400196BE40864204D1019BDE0777
:10BC9000F60F02239B1B0E46164318D1002D16DA11
:10BCA000002C03D0022B01D0012B06D00220FEF77E
:10BCB00077FEFEF73BFE1BB0F0BD0220FEF770FEE4
:10BCC000FEF734FE0122D20751401BB0F0BD039EA7
:10BCD000002E61D1BF4EB04220D1C148844201D173
:10BCE000002A08D0B948814209DB002D10DB1898E2
:10BCF00029461BB0F0BD0020B4491BB0F0BD002D9B
:10BD000006DA01222946D207189851401BB0F0BD2F
:10BD1000B4497944086849681BB0F0BDAB4FB842DC
:10BD200025D1002D1FDA002904D0B14212D1002AFA
:10BD300009D018E0002A72D1A649E20F0020D207EC
:10BD400011431BB0F0BD0020E20F0146D2071143A2
:10BD50001BB0F0BDB14206DA234600203946F9F7A0
:10BD6000FBFB1BB0F0BD104621461BB0F0BDB1423D
:10BD700012DA0126B607B54203D12346104619460A
:10BD8000FEE3994EB54207D1261E05DB104631462B
:10BD900000F040FC1BB0F0BD67007F081646002A8B
:10BDA00040D100290AD08B4A914229D1002C0EDDC6
:10BDB000002D1CDB002011461BB0F0BD022B16D05D
:10BDC000002C14D0012B12D1002C14DB0FE0002C1E
:10BDD00028DA002D09DB012B03D000207D491BB0A0
:10BDE000F0BD002081491BB0F0BD012B03D0002025
:10BDF00001461BB0F0BD00200121C9071BB0F0BDFA
:10BE0000724A91420ED1002C01DA002B17D0022B7E
:10BE100006D00020C043F9F73FFC1BB0F0BD90E214
:10BE20000120F8E7E217521C94461A4307D000227B
:10BE30000892664C62465B1E1A4307D009E0012057
:10BE4000FEF7AEFDFEF780FD1BB0F0BD0022644C96
:10BE50000892674A90427DDD664B674A98421FDD33
:10BE6000914202DC002D05DB4DE05848814217DB92
:10BE7000002D48DD0220FEF793FDFEF76DFD05461F
:10BE80000E460022534B21460898F9F7FDFA084662
:10BE900071004908C00FC007014328461BB0F0BD20
:10BEA000914215DA002D2EDA0220FEF779FDFEF719
:10BEB00053FD05460E460022464B21460898F9F7E9
:10BEC000E3FA72005208C80FC0070243114617E098
:10BED0003E4B994223DD002D15DD0220FEF760FD6B
:10BEE000FEF73AFD05460E4600223A4B21460898D9
:10BEF000F9F7CAFA084671004908C00FC0070143A4
:10BF000028461BB0F0BD0220FEF74AFDFEF72EFDCD
:10BF100049004908E20FD20711431BB0F0BD0022CF
:10BF200030463946F9F7A2FA012205460E46D243B9
:10BF3000F9F78AFB314A324BF9F79EFA2A46334623
:10BF4000F9F7A2FA0022284BF9F796FA07462A4693
:10BF5000334600E064E0039110461946F9F794FA7D
:10BF60003A46039BF9F790FA0746032209915207D4
:10BF7000244B28463146F9F787FA07910C90224A5C
:10BF8000204B38460999F9F77FFA074601911F4A75
:10BF90001F4B28463146F9F777FA3A46019BF9F7E5
:10BFA00065FA07460B460246099107990C98F9F77E
:10BFB000B9F900250E462846079B0C9AF9F756FA60
:10BFC0003A4627E0FFFF1F00FFFF0F000000F03F91
:10BFD0000000E0FF0000F07F0000404301FCFFFF95
:10BFE0000000F0BF5A0B00000000E03F0000F0FF2F
:10BFF0000000E0410000F043FFFFEF3F555555556D
:10C000005555D53F4715F73FFE822B6544DF5DF858
:10C010000BAE543E099BF9F72FFA02460B4652E14C
:10C02000012500202D05A94207DA35223046394680
:10C03000F9F70AFB06463420C0430A151218FE48D9
:10C04000101803900803FD49000B01430F46FC49FB
:10C05000884201DC002003E0FA49884202DA01202C
:10C06000119005E0002011900398401C7F1B039065
:10C0700011980597C200F4480F92784480184368DD
:10C080000268394630460D930292F9F7EFF90791AD
:10C090000C9030460D9B029A0599F9F743F9024638
:10C0A0000B460020E549F9F757FA09910490079BE0
:10C0B0000C9AF9F7E9F9129000201090E3480D4628
:10C0C000784400680E9001217810490708431199BF
:10C0D0000D9B890440180121C90447183946029A6A
:10C0E0000E98F9F7C3F93246059BF9F7C5F90246F0
:10C0F0000B4629461098F9F7C7F9064602913B46C8
:10C1000029460E9A1098F9F7BFF9079B0C9AF9F790
:10C11000B3F93246029BF9F7A9F9099B049AF9F79A
:10C12000B3F90591129A0A902B4610461946F9F771
:10C13000ABF906460246C6480F460B460621784430
:10C14000FEF79EFB32463B4600910490104619468E
:10C15000F9F79AF9009B049AF9F796F906460F4603
:10C160002B461946129A1098F9F7DCF8059B0A9AA3
:10C17000F9F78AF932463B46F9F7D4F8109A079155
:10C1800004902B4610461946F9F77EF9B14E00226D
:10C19000334609910290F9F7C5F8079B049AF9F71D
:10C1A000C1F800200746024633460091F9F75EF9D0
:10C1B000099B029AF9F75AF9079B049AF9F75CF977
:10C1C00006460D913A462946009B1098F9F75CF90E
:10C1D00007910C902B463046129A0D99F9F754F9B5
:10C1E00005460E463A46009B05990A98F9F74CF920
:10C1F00033462A46F9F796F802460B460746099158
:10C2000007990C98F9F78EF800250E462846079BEB
:10C210000C9AF9F72BF93A46099BF9F72DF90746DD
:10C220000722099152078C4B31462846F9F72CF921
:10C2300007910090894A884B38460999F9F724F903
:10C2400007460191864A874B31462846F9F71CF983
:10C250003A46019BF9F766F8834B7B440F9A9B188B
:10C260001A685B68F9F75EF8029009910398F9F78C
:10C2700013FA05910490099B029A07990098F9F71F
:10C2800051F87A4B7B440F9A9B181A685B681746E3
:10C290000393F9F747F8059B049AF9F743F80E461C
:10C2A0002846059B049AF9F7E1F83A46039BF9F70B
:10C2B000DDF8079B009AF9F7D9F8099B029AF9F77C
:10C2C000DBF802460B46199900200C900F4618988F
:10C2D000F9F7DAF8029104903B460C9A19991898EC
:10C2E000F9F7C4F82A463346F9F7CEF8029B049AC8
:10C2F000F9F718F809910E902A46334639460C98FA
:10C30000F9F7C2F806460F46099B0E9AF9F70AF8A4
:10C31000574A0D46914220DB5242AA18024310D1DF
:10C3200032463B46F9F7A2F804900391514A524B2A
:10C3300009990E98F8F7F6FF039B049AF9F74CFA5F
:10C340001ED20220FEF72CFBFEF706FB490049082F
:10C35000E20FD20711431BB0F0BD6A00474B5208F1
:10C360009A420DD3464AAA18024300D0CBE5324682
:10C370003B46F9F77BF8099B0E9AF9F72DFAF5D9A8
:10C380006800002340082C490393020D3D4B5218CE
:10C39000984223DD01200005521CD0404219500074
:10C3A000400D401838497944096813468C4637498E
:10C3B000C1408B4312030121120B090551181422AD
:10C3C000101AC1400391002D01DA484203906246E1
:10C3D00030463946F9F74AF806460F4632463B469C
:10C3E00009990E98F8F79EFF00252A46284B284603
:10C3F0000591F9F749F807910C90264A264B2846F3
:10C400000599F9F741F80091029032463B462846DB
:10C410000599F9F72BF8099B0E9AF9F72DF81F4AA1
:10C420001F4BF9F731F8009B029AF8F77BFF07469C
:10C430000B460246099135E001FCFFFF0000F03F8A
:10C440008E9803007AB60B006A070000AC07000064
:10C45000D60600000000084009C7EE3FFD033ADCA5
:10C46000F5015B14E02F3EBEAA0500007005000038
:10C4700000009040FE822B654715973C00CC904011
:10C4800000346F3F0000E03FC6040000FFFF0F00D4
:10C49000432EE63F396CA80C615C20BEEF39FAFEF2
:10C4A000422EE63F07990C98F8F73CFF05460E46EA
:10C4B000079B0C9AF8F7DAFF3A46099BF8F7DCFF7E
:10C4C00009912A4633460E9010461946F8F7DCFFCC
:10C4D000074602462F480B46059105217844FEF792
:10C4E000CFF93A46059BF8F7CFFF2A463346F8F7CF
:10C4F000C3FF0746019128463146099B0E9AF8F77B
:10C50000C3FF099B0E9AF8F70DFF012304910C90CD
:10C5100000229B0738460199F8F7A8FF05910E9075
:10C520003A4628463146019BF8F7AEFF059B0E9A26
:10C53000F9F712F8049B0C9AF8F798FF2A4633464D
:10C54000F8F794FF0022144BF8F796FF064603987D
:10C550000D46000541190915002912DC304629460F
:10C56000039AF9F771F8FEF745F9042801D1FEF7AF
:10C57000FDF930462946039AF9F766F8064601E0C8
:10C5800004E029180B46324621460898F8F77CFF4C
:10C590001BB0F0BD680300000000F03FF0B58C4612
:10C5A00000251026052109078E620E4C08E067461B
:10C5B0007F5DE760A768FF07FCD0E7681F706D1C10
:10C5C0008542F4DB0020074606E0E760A568ED073A
:10C5D000FCD0E5681D54401C9042F6D38E610020CB
:10C5E000F0BD00000030014070B572B60124074D67
:10C5F000A40221462846F9F7E7FC002804D0224689
:10C6000003492846F9F784FD62B670BD00FC0008B6
:10C61000C80D0020F8B506460C46F9F7EBF9051EE3
:10C620000F4600D00120014349000B484908411A38
:10C63000C90F0DD0002E01D0012100E000210C43D4
:10C6400061004908401AC00F02D10120FEF7A8F985
:10C6500028463946F8BD00000000F07FF8B51546C1
:10C660000E460746002407E03819C0B200F008F86B
:10C67000641C2870E4B26D1CB442F5D33046F8BD9A
:10C6800010B50446FCF716F8EE20FBF7E6FFFCF7C2
:10C690004AF82046FBF7E1FFFCF745F8FCF70AF8FB
:10C6A000EF20FBF7DAFFFCF73EF80020FBF7A8FFCE
:10C6B0000446FCF71AF8204610BD704770B50D46C9
:10C6C0000446FBF7F7FFEE20FBF7C7FFFCF72BF85C
:10C6D0002046FBF7C2FFFCF726F82846FBF7BDFF14
:10C6E000FCF721F8FCF701F80A20FEF7A2FA70BD6A
:10C6F000F0B50025102605279C463F070B46BE6275
:10C700000C4C06E0595DE160A168C907FCD0E16806
:10C710006D1C8542F6DB002007E06146095CE160A4
:10C72000A168C907FCD0E168401C9042F5D3BE6106
:10C730000020F0BD003001400000010203040005AC
:10C74000405C0000A05C0400C06C0800805C040039
:10C75000E03F1E00E07D1E0007A9022570889B882F
:10C760000A001600010006000100020087008D008B
:10C770002D001A3152001A339A001A351D011A374A
:10C780006B003B31BE003B335E013B3596023B37CD
:10C79000000099599959EB518F421E45142E008083
:10C7A000EB51F5283333E13A703DE13AC235852B40
:10C7B000C2353333C235C235AE47E13A5138A330C2
:10C7C00051380000000000000000010203040607C9
:10C7D0000809030406080C101820300000000001AE
:10C7E0000203040000000000000000000000F03F11
:10C7F000000000000000F83F000000000000000002
:10C800000000004003B8E23F00000000000000000C
:10C8100006D0CF43EBFD4C3E033333333333E33F9A
:10C82000FFAB6FDBB66DDB3F4D268F515555D53FC6
:10C8300001411DA96074D13F65DBC9934A86CD3F94
:10C84000EF4E454A287ECA3F3E5555555555C53F82
:10C8500093BDBE166CC166BF2CDE25AF6A56113F74
:10C86000F16BD2C541BDBBBED0A4BE726937663E76
:10C87000000000000000000098C800080000002030
:10C8800070010000BC5A0008DCC8000870010020DC
:10C89000001B000090A900080124130704380D09AB
:10C8A0001E080540082609104008560A131D043BBF
:10C8B00008BE0516D8BC4010085201033CC8420708
:10C8C0007652030CE5800C140202141509090102CA
:0CC8D000628149D0013A29409204922074
:04000005080050C1DE
:00000001FF
